:0400000057EF00F0C6
:10000800AE5BAE5BAE5BAE5BAE5BAE5BAE5BAE5BA0
:10001800E359AE5BAE5BAE5BAE5BAE5BAE5BAE5B5D
:10002800AE5BAE5BAE5BAE5BAE5BAE5BAE5BAE5B80
:10003800AE5BAE5BAE5BC655AE5BAE5BAE5B3D58D2
:10004800AE5BAE5BAE5BAE5B2B00AE5BAE5BAE5B3E
:10005800AE5BAE5BAE5BAE5BAE5BAE5BAE5BAE5B50
:10006800AE5BAE5BAE5BAE5BAE5BAE5BAE5BAE5B40
:10007800AE5BAE5B2B00AE5BAE5BAE5B2B002B00CA
:100088002B002B002B002B002B002B00AE5BAE5B54
:100098009C59AE5BAE5BAE5B2B002B002B002B009C
:0A00A800AE5BAE5BFF0025EFACF08D
:10F800000000000000001B1B0000181818181B1B2C
:10F810000000030303031B1B00001B1B1B1B1B1B04
:10F8200000040E1F0404040400040404041F0E0456
:10F83000001112140B110203000E0A0E000000004A
:10F8400000086E01D26901246D011E49017856013C
:10F850008A5A01D45501FA6D01AA6E01A66E01D42F
:10F860006A014E6E01566E01EC6D01466E01CE6D61
:10F8700001385E01FA5B01BE6D010080C094D420A6
:10F880002000204861726477617265203A2042410D
:10F8900053452031384632374B3432202B20493201
:10F8A00043204C434434783230202B2052544320A0
:10F8B000445333323331202B2055415254312031BF
:10F8C00031353230300D0A20536368656D613A205E
:10F8D000536368E96D615F506F727461696C5F5664
:10F8E000352D302D312064752031302D30332E7080
:10F8F000646620627920482E542E0D0A0D0A0020DD
:10F90000417574726573203A0D0A20204C43445FA0
:10F9100034626974735F4932435F323032342D3060
:10F92000312C2055415254315F46756E6374696FB6
:10F930006E732E68202C206D63632E682C0D0A00D8
:10F9400045434F2E2E2E2E0042415252455F470016
:10F9500042415252455F44004241525245474400A1
:10F96000464C454348204800464C4543485F4200CA
:10F97000312F324865757200444547524543200097
:10F98000204C43445F63686172735F5370656369C1
:10F990006175785F323032342E682C202020456526
:10F9A00070726F6D203A20456570726F6D2E2E2E2D
:10F9B0002E2E2E2E2E2E2E2E2020200D0A002052EE
:10F9C00041303D2E2E2E5241313D416E616C6F67AC
:10F9D000202C5241343D6C65642C5241332E2E2E26
:10F9E0005243363D545820554152543120524337EA
:10F9F0003D525820554152540D0A00204120696E55
:10FA0000636C7572653A200D0A204469616C6F67FA
:10FA100075655F4F70657261746575725F50435FA5
:10FA20007669615F554152545F323032332D30393F
:10FA300030350D0A0D0A00204469726563746F72D7
:10FA400079203A433A5C4D504C4142585F50726FB6
:10FA50006A656374735C31384632374B34325F50B9
:10FA60004D575F434350313233345F323032350DBE
:10FA70000A0020424153452031384632374B343258
:10FA8000202B204C4344345832302B2050574D31DA
:10FA90002C322C332C3420416E616C6F6720524124
:10FAA000302C312C322C330D0A00204C43442034AE
:10FAB0007832302062757320493243312048572014
:10FAC0003A205243333D53434C2C5243343D53442C
:10FAD000410D0A002050726F6A656374203A20312C
:10FAE000384632374B34325F504D575F43435031C5
:10FAF0003233345F323032350D0A0020536F757265
:10FB00006365203A20206D61696E2E63202C20727F
:10FB10006576203A5F3235303331370D0A002043A5
:10FB20006F6E6669672020496E7465726E616C2025
:10FB3000466F73632036344D487A0D0A002020202A
:10FB400020202020202020202020202020202020B5
:10FB5000200020524230202E2E2E0D0A002052610D
:10FB60007070656C203A2063646520504D57793D74
:10FB700058585858206176656320793D63686F69ED
:10FB80007820504D5720312061203420657420208A
:10FB900078787878202076616C6575722064757449
:10FBA000792030303030206120313031350D0A007D
:10FBB000205465737420646966666572656E746549
:10FBC000732076616C65757273206465204475746A
:10FBD000792D6379636C6520766961206C6520639B
:10FBE0006C6176696572207465726D696E616C20F6
:10FBF000594154200D0A0020496E697469616C698D
:10FC0000736174696F6E2050574D312C322C332C38
:10FC1000342061766563204652657120332C394B60
:10FC2000487A202854696D6572322C54696D65726A
:10FC300034290D0A00456E7472657220756E652058
:10FC400076616C6575722050574D3D7878787820D4
:10FC500070756973203C656E7465723E2061752015
:10FC6000636C61766965720D0A002076657273694E
:10FC70006F6E2050726F746F74797065203A204CEB
:10FC8000434420426C65752061206C276164726575
:10FC9000737365203078323720210D0A00204572B9
:10FCA00072657572206465205361697369652020EF
:10FCB00063686F6978204343502025632076616C28
:10FCC0006575722050574D202535640D0A00200DB2
:10FCD0000A53657175656E6365206427496E6974A2
:10FCE000204C4344203478323020766961204932F8
:10FCF000433120504346383537340D0A0020402028
:10FD0000646563696D616C20232534752020736FF1
:10FD1000697420404465766963652037626974734D
:10FD2000203D203058253032582000204368617231
:10FD300067656D656E742063617261637465726579
:10FD4000732053706563696175782020656E204368
:10FD50004752414D0D0A0020436F6D70696C656418
:10FD6000202573206174202573205554432020766C
:10FD7000657273696F6E20584338203A2564200DF0
:10FD80000A0020546573742070726573656E636534
:10FD9000206465766963657320737572204275739C
:10FDA00020493243310D0A00206164726573736526
:10FDB000204C43443D20256420736F6974203058E3
:10FDC00025303258200D0A00202A2050574D31206E
:10FDD000737572205243322028544D5232293D32DD
:10FDE0003025200D0A00202A2050574D32207375EF
:10FDF00072205243312028544D5232293D3430254F
:10FE0000200D0A00202A2050574D33207375722090
:10FE10005242302028544D5234293D363025200D91
:10FE20000A00202A2050574D342073757220524208
:10FE3000352028544D5234293D383025200D0A00F4
:10FE4000456570726F6D2032344C4378787820327B
:10FE500035366B206F75203531324B0020504346CC
:10FE60003837353420666F72204C43442032783165
:10FE700036636172730020496E69745F49324328AA
:10FE800029203130304B687A3B0D0A0043617261A2
:10FE9000637465726573205370656369617578205A
:10FEA0000050574D342D52423020253464202533E4
:10FEB0002E316625630050574D322D524331202597
:10FEC00034642025332E3166256300504D57322D82
:10FED000524331202534642025332E3166256300BA
:10FEE00050574D312D524332202534642025332E76
:10FEF000316625630050574D332D5242352025344D
:10FF0000642025332E3166256300205072657320EE
:10FF1000456E746572206B657920210D0A00566567
:10FF20007273696F6E2050726F746F747970652090
:10FF300021005043463835373441203862697473A4
:10FF400020492F4F002050726573656E746174698B
:10FF50006F6E203A0D0A004C434420323131392073
:10FF60003278313663617273005043463835373426
:10FF700020386269747320494F00454550524F4DF7
:10FF8000203531326279746573002045727265756F
:10FF9000722063780D0A004F4C454420535344317E
:10FFA000333036006E6F6E20726563656E73E900E4
:10FFB00020536169736965204F4B20004D617220A9
:10FFC00031372032303235005254432044533332DB
:10FFD00033310031303A34303A3031005265637594
:10FFE000203A00494E46004E414E00696E66006E52
:0FFFF000616E006C6C7300202E31006C66000097
:020000040001F9
:1000000041ECB5F0000E0001EF6F000EE86F000E3E
:10001000E76F000EE725D96E030EE821DA6E000EB9
:10002000DF6EE74BE82BE85109E1800EE75DD8A0D1
:100030001CEF80F01EEF80F009EF80F0000EE86FFB
:10004000000EE76F800EE725D96E030EE821DA6E09
:10005000000EDF6EE74BE82BE85109E1800EE75D0B
:10006000D8A035EF80F037EF80F022EF80F0000E5F
:10007000E86F000EE76F200EE725D96E020EE8212B
:10008000DA6E000EDF6EE74BE82BE85109E17F0ED8
:10009000E75DD8A04EEF80F050EF80F03BEF80F0AE
:1000A000000EE86F000EE76F2A0EE725D96E010EED
:1000B000E821DA6E000EDF6EE74BE82BE85109E12C
:1000C000090EE75DD8A067EF80F069EF80F054EF8C
:1000D00080F0000EE16F030EE26FBCECB2F0D9ECE1
:1000E000ABF0000E0001E86F000EE76FBA88110E4A
:1000F0000101F06F3C0EEF6FCB0EE82EFED7EF2F15
:10010000FCD7F02FFAD7BA98110E0101F06F3C0E10
:10011000EF6FCB0EE82EFED7EF2FFCD7F02FFAD7DC
:100120000001E74BE82BE85109E1080EE75DD8A094
:100130009CEF80F09EEF80F076EF80F0BA88CAECFA
:10014000B1F0090E0101F06F1E0EEF6FE40EE82E04
:10015000FED7EF2FFCD7F02FFAD700F0BBECB4F0AE
:10016000BBECB4F0450E046EFF0E056ED3ECB0F0A0
:10017000000E0001E86F000EE76FD890E735D96EEA
:10018000E835DA6ED00ED926010EDA226F0078FF3C
:1001900004F06F0074FF05F0D3ECB0F00001E74B02
:1001A000E82BE85109E1090EE75DD8A0DAEF80F00D
:1001B000DCEF80F0BDEF80F0BBECB4F0E1C0B6F056
:1001C000E2C0B7F0570E0001B86FFD0EB96FBC0E5C
:1001D000BA6FFF0EBB6FD30EBC6FFF0EBD6F090E63
:1001E000BF6F380EBE6FFEECB0F0E1C004F0E2C0AD
:1001F00005F0E4ECAEF0BBECB4F0020EFCECB2F0B7
:100200006A0E046EFC0E056ED3ECB0F0760E046E32
:10021000FE0E056ED3ECB0F0B5ECB5F0820E046EB8
:10022000FD0E056ED3ECB0F087EC9BF0BBECB4F0A8
:10023000270E5B6E000E0001FB6F140EFA6F200E8E
:10024000B66F020EB76FA80EB86FFD0EB96F5BC028
:10025000BAF0BB6B5BC0BCF0BD6BFEECB0F0200E27
:10026000046E020E056EE4ECAEF03D017589CE0E13
:10027000046EFC0E056ED3ECB0F03D01738FF4EC10
:10028000A3F0BBECB4F0010E6FECACF0010E2B6EE2
:100290001E0E2C6EFF0E2D6E010E49ECB6F0020EF6
:1002A000FCECB2F0010E6FECACF0020E6FECACF0B7
:1002B000090E0101F06F1E0EEF6FE40EE82EFED75F
:1002C000EF2FFCD7F02FFAD700F02B0E046EFD0EA7
:1002D000056ED3ECB0F08C0E246EFE0E256E00EC95
:1002E000ADF0000E276E000E266E55ECA3F0000E4A
:1002F0000001E86F000EE76F000E276E020E266EFB
:10030000010EE725286E000EE821296EE7C02AF0CD
:10031000F6ECA7F00001E74BE82BE85109E1080EE5
:10032000E75DD8A096EF81F098EF81F07CEF81F047
:10033000010EFCECB2F0F70E046EFB0E056ED3EC72
:10034000B0F07AECB6F06EECB6F062ECB6F056ECCB
:10035000B6F0BBECB4F0C2ECADF0D28ED28EC80ECB
:10036000046EFD0E056ED3ECB0F0E60E046EFD0ECD
:10037000056ED3ECB0F0040E046EFE0E056ED3ECE9
:10038000B0F0220E046EFE0E056ED3ECB0F0010E3E
:100390006FECACF0020E6FECACF0000E5A6EC80EB3
:1003A000596E59C004F05AC005F0066A076A000E7B
:1003B000C9EC9EF004C012F005C013F006C014F0A2
:1003C00007C015F0330E166E330E176E230E186E1F
:1003D000410E196EF2EC96F012C05CF113C05DF1A3
:1003E00014C05EF115C05FF159C004F05AC005F0A9
:1003F00043ECB4F0200E0001B66F020EB76FE00EB2
:10040000B86FFE0EB96F59C0BAF05AC0BBF05CC1EC
:10041000BCF05DC1BDF05EC1BEF05FC1BFF0000EBB
:10042000C16F250EC06FFEECB0F0010E2B6E200EDA
:100430002C6E020E2D6E010E3CECB6F0010E5A6EC3
:10044000900E596E59C004F05AC005F0066A076A4A
:10045000000EC9EC9EF004C012F005C013F006C0F7
:1004600014F007C015F0330E166E330E176E230E00
:10047000186E410E196EF2EC96F012C058F113C0CE
:1004800059F114C05AF115C05BF159C004F05AC0BB
:1004900005F043ECB4F0200E0001B66F020EB76F0A
:1004A000B60EB86FFE0EB96F59C0BAF05AC0BBF0A5
:1004B00058C1BCF059C1BDF05AC1BEF05BC1BFF01C
:1004C000000EC16F250EC06FFEECB0F0010E2B6E5A
:1004D000200E2C6E020E2D6E020E3CECB6F0020EBB
:1004E0005A6E580E596E59C004F05AC005F0066A8B
:1004F000076A000EC9EC9EF004C012F005C013F0AC
:1005000006C014F007C015F0330E166E330E176ECA
:10051000230E186E410E196EF2EC96F012C054F1D3
:1005200013C055F114C056F115C057F159C004F06D
:100530005AC005F043ECB4F0200E0001B66F020E75
:10054000B76FF50EB86FFE0EB96F59C0BAF05AC04A
:10055000BBF054C1BCF055C1BDF056C1BEF057C18F
:10056000BFF0000EC16F250EC06FFEECB0F0010EA3
:100570002B6E200E2C6E020E2D6E030E3CECB6F090
:10058000030E5A6E200E596E59C004F05AC005F081
:10059000066A076A000EC9EC9EF004C012F005C09E
:1005A00013F006C014F007C015F0330E166E330EAC
:1005B000176E230E186E410E196EF2EC96F012C0F3
:1005C00050F113C051F114C052F115C053F159C08C
:1005D00004F05AC005F043ECB4F0200E0001B66FF1
:1005E000020EB76FA10EB86FFE0EB96F59C0BAF008
:1005F0005AC0BBF050C1BCF051C1BDF052C1BEF0F9
:1006000053C1BFF0000EC16F250EC06FFEECB0F0FD
:10061000010E2B6E200E2C6E020E2D6E040E3CEC85
:10062000B6F0B00E046EFB0E056ED3ECB0F0350ED6
:10063000046EFC0E056ED3ECB0F0C2ECADF07A0E99
:100640000101F06FC10EEF6F810EE82EFED7EF2F84
:10065000FCD7F02FFAD700D00001F405D8A433EF6F
:1006600083F035EF83F071EF86F0DC0E046EFF0E41
:10067000056ED3ECB0F0800E046E030E056EE4EC54
:10068000AEF0BBECB4F0800E0001DF6F030EE06F44
:1006900060007FF3D9FF600083F3DAFF500EDE18AD
:1006A000D8A455EF83F057EF83F06AEF86F020EE81
:1006B00001F0DF51D926E051DA22570EDE18D8A416
:1006C00064EF83F066EF83F06AEF86F020EE02F0CD
:1006D000DF51D926E051DA224D0EDE18D8A473EF8F
:1006E00083F075EF83F06AEF86F020EE04F0DF51BF
:1006F000D926E051DA223D0EDE18D8A482EF83F02D
:1007000084EF83F06AEF86F020EE03F0DF51D92604
:10071000E051DA22DF50F66F000EE66F000EE56F53
:10072000D00E0101EF6FFF0EF06F0001F6510101D5
:10073000F16FF26BEF51F127F051F223F25107E123
:100740000A0EF15DD8B0A7EF83F0A9EF83F06AEF4E
:1007500086F0300E0001F665B0EF83F0B2EF83F063
:100760006AEF86F0350EF661B8EF83F0BAEF83F0EA
:100770006AEF86F0E54BE62BD00E0101EF6FFF0E1E
:10078000F06F000120EE05F0DF51D926E051DA22AA
:10079000DF500101F16FF26BEF51F127F051F223BD
:1007A000F25107E10A0EF15DD8B0D9EF83F0DBEF2B
:1007B00083F0F8EF83F0000120EE05F0DF51D92639
:1007C000E051DA22DF500101EF6FD00EEF25046E09
:1007D000056AFF0E0522030E076EE80E066E2CEC6E
:1007E000B5F004C059F005C05AF00001E54BE62B06
:1007F000D00E0101EF6FFF0EF06F000120EE06F04A
:10080000DF51D926E051DA22DF500101F16FF26B9E
:10081000EF51F127F051F223F25107E10A0EF15D99
:10082000D8B015EF84F017EF84F036EF84F00001B4
:1008300020EE06F0DF51D926E051DA22DF50010127
:10084000EF6FEF51640D6F00CCFFF0F16F00D0FF40
:10085000F1F15950F0275A50F123400EF025596E0E
:10086000ED0EF1215A6E0001E54BE62BD00E010191
:10087000EF6FFF0EF06F000120EE07F0DF51D92679
:10088000E051DA22DF500101F16FF26BEF51F127F5
:10089000F051F223F25107E10A0EF15DD8B053EFA7
:1008A00084F055EF84F074EF84F0000120EE07F03F
:1008B000DF51D926E051DA22DF500101EF6FEF510D
:1008C0000A0D6F00CCFFF0F16F00D0FFF1F159502D
:1008D000F0275A50F123200EF025596EFE0EF1211B
:1008E0005A6E0001E54BE62BD00E0101EF6FFF0EB3
:1008F000F06F000120EE08F0DF51D926E051DA2236
:10090000DF500101F16FF26BEF51F127F051F2234B
:10091000F25107E10A0EF15DD8B091EF84F093EF48
:1009200084F0ACEF84F0000120EE08F0DF51D9260E
:10093000E051DA22DF500101EF6FEF515924F06FDF
:10094000000E5A20F16FD00EF025596EFF0EF121E6
:100950005A6E0001E54BE62B050E0001E519E61184
:10096000D8A4B5EF84F0B7EF84F04DEF86F0F80E21
:10097000595C030E5A58D8B0C0EF84F0C2EF84F02F
:100980004DEF86F0BC8A12EF86F0B00E046EFF0EBB
:10099000056ED3ECB0F059C004F05AC005F0066AF9
:1009A000076A000EC9EC9EF004C012F005C013F0F7
:1009B00006C014F007C015F0330E166E330E176E16
:1009C000230E186E410E196EF2EC96F012C05CF117
:1009D00013C05DF114C05EF115C05FF1200E00017F
:1009E000B66F020EB76FE00EB86FFE0EB96F59C04A
:1009F000BAF05AC0BBF05CC1BCF05DC1BDF05EC1D5
:100A0000BEF05FC1BFF0000EC16F250EC06FFEECDF
:100A1000B0F0010E2B6E200E2C6E020E2D6E010E0C
:100A20003CECB6F059C004F05AC005F043ECB4F009
:100A300030EF86F059C004F05AC005F0066A076A24
:100A4000000EC9EC9EF004C012F005C013F006C001
:100A500014F007C015F0330E166E330E176E230E0A
:100A6000186E410E196EF2EC96F012C058F113C0D8
:100A700059F114C05AF115C05BF1200E0001B66F98
:100A8000020EB76FCB0EB86FFE0EB96F59C0BAF039
:100A90005AC0BBF058C1BCF059C1BDF05AC1BEF03C
:100AA0005BC1BFF0000EC16F250EC06FFEECB0F051
:100AB000010E2B6E200E2C6E020E2D6E020E3CECE3
:100AC000B6F059C004F05AC005F02BECB4F030EF8A
:100AD00086F059C004F05AC005F0066A076A000E95
:100AE000C9EC9EF004C012F005C013F006C014F06B
:100AF00007C015F0330E166E330E176E230E186EE8
:100B0000410E196EF2EC96F012C054F113C055F17B
:100B100014C056F115C057F1200E0001B66F020E39
:100B2000B76FF50EB86FFE0EB96F59C0BAF05AC064
:100B3000BBF054C1BCF055C1BDF056C1BEF057C1A9
:100B4000BFF0000EC16F250EC06FFEECB0F0010EBD
:100B50002B6E200E2C6E020E2D6E030E3CECB6F0AA
:100B600059C004F05AC005F013ECB4F030EF86F031
:100B700059C004F05AC005F0066A076A000EC9ECB5
:100B80009EF004C012F005C013F006C014F007C0B8
:100B900015F0330E166E330E176E230E186E410EBF
:100BA000196EF2EC96F012C050F113C051F114C05E
:100BB00052F115C053F1200E0001B66F020EB76F4F
:100BC000A10EB86FFE0EB96F59C0BAF05AC0BBF093
:100BD00050C1BCF051C1BDF052C1BEF053C1BFF015
:100BE000000EC16F250EC06FFEECB0F0010E2B6E33
:100BF000200E2C6E020E2D6E040E3CECB6F059C089
:100C000004F05AC005F0FBECB3F030EF86F0000EB4
:100C10000001F66F8A0E046EFF0E056ED3ECB0F085
:100C200030EF86F0F6510101EF6FF06BF051000AE2
:100C3000D8B41DEF86F007EF86F0EF51310AD8B433
:100C4000C5EF84F0030AD8B41AEF85F0010AD8B4CE
:100C500069EF85F0070AD8B4B8EF85F007EF86F0A2
:100C60000001F651D8B437EF86F039EF86F04AEF3D
:100C700086F0200E046E020E056EE4ECAEF0BBECC6
:100C8000B4F0D00E0101EF6FC90EE82EFED7EF2FA2
:100C9000FCD700D0BC9A6AEF86F0200EB66F020E29
:100CA000B76F9D0EB86FFC0EB96FF6C0BAF0BB6B94
:100CB00059C0BCF05AC0BDF0FEECB0F0200E046E7E
:100CC000020E056EE4ECAEF05D0E046EFB0E056EDA
:100CD000D3ECB0F0000E0001DF6F000EE06F000EED
:100CE000F46FBC8A090E0101F06F1E0EEF6FE40E67
:100CF000E82EFED7EF2FFCD7F02FFAD700F0BC9AE2
:100D000017EF83F057EF00F0000E0001756F000E33
:100D1000746F41C086F042C087F043C088F044C081
:100D200089F089BF98EF86F096EF86F0AEEF86F0F7
:100D3000000E756F010E746F86C004F087C005F059
:100D400088C006F089C007F08EECB3F004C086F0CE
:100D500005C087F006C088F007C089F0000E0001CA
:100D60008D6F000E8C6FD5C078F0D6C079F07451BD
:100D70007511D8A4BEEF86F0C0EF86F0C7EF86F0FD
:100D8000D9A5C5EF86F0C7EF86F0E1EF86F0745184
:100D90007511D8A4CEEF86F0D0EF86F0D6EF86F0AE
:100DA000000E616F2B0E606FDAEF86F0000E616F40
:100DB0002D0E606F60C080F18C4B8D2B7807D8A012
:100DC000790786C004F087C005F088C006F089C0A6
:100DD00007F027ECA6F004040510D8A4F2EF86F083
:100DE000F4EF86F03FEF87F0BF0E466EFF0E476EC2
:100DF0004550486E496A4650482647504922495056
:100E000007E11A0E485CD8B008EF87F00AEF87F0C8
:100E100019EF87F0800E00018C25086E010E8D21E0
:100E2000096EE30E0A6EFF0E0B6E88ECAFF026EF34
:100E300087F0800E00018C25086E010E8D21096E51
:100E4000EB0E0A6EFF0E0B6E88ECAFF00001FD0E8C
:100E50007827FF0E79233FC014F040C015F0800EB4
:100E6000166E010E176E78C018F079C019F0CAEC32
:100E7000A8F014C03FF015C040F08CEF8CF086C095
:100E800004F087C005F088C006F089C007F027ECA1
:100E9000A6F004500510D8A450EF87F052EF87F069
:100EA00086EF87F0BF0E466EFF0E476E4550486EC8
:100EB000496A4650482647504922495007E11A0ED0
:100EC000485CD8B066EF87F068EF87F077EF87F07F
:100ED000800E00018C25086E010E8D21096EE70E33
:100EE0000A6EFF0E0B6E88ECAFF026EF87F0800ED7
:100EF00000018C25086E010E8D21096EEF0E0A6E21
:100F0000FF0E0B6E88ECAFF026EF87F0000E0001AD
:100F10008E6F000E8F6F800E906F3F0E916F000EE0
:100F20008B6F000E8A6F86C004F087C005F088C002
:100F300006F089C007F0000E086E000E096E000E64
:100F40000A6E000E0B6E43ECAAF0D8B0AAEF87F041
:100F5000ACEF87F02FEF88F0CBEF87F08EC004F076
:100F60008FC005F090C006F091C007F0000E086E2B
:100F7000000E096E200E0A6E410E0B6ECBEC94F043
:100F800004C08EF005C08FF006C090F007C091F04D
:100F900000018A4B8B2B86C01DF087C01EF088C0D5
:100FA0001FF089C020F0000E086E000E096E200EA2
:100FB0000A6E410E0B6E8EC004F08FC005F090C01B
:100FC00006F091C007F0CBEC94F004C021F005C00E
:100FD00022F006C023F007C024F0A5ECA5F0D8B09D
:100FE000F4EF87F0F6EF87F0AEEF87F016EF88F0BA
:100FF0008EC012F08FC013F090C014F091C015F0A5
:10100000000E166E000E176E200E186E410E196E31
:10101000F2EC96F012C08EF013C08FF014C090F076
:1010200015C091F000018A07D8A08B0786C01DF07B
:1010300087C01EF088C01FF089C020F08EC021F04C
:101040008FC022F090C023F091C024F0A5ECA5F051
:10105000D8A02DEF88F02FEF88F0F8EF87F045C08B
:101060000AF00B6AEEECB1F00A5000017B6F7BC016
:101070007AF0670E7B19D8A440EF88F042EF88F031
:1010800068EF88F0D751D811D8A449EF88F04BEF1A
:1010900088F04FEF88F0000ED86F010ED76FD8BFE1
:1010A0005CEF88F0D85106E1D705D8B05AEF88F048
:1010B0005CEF88F062EF88F0000E776F060E766FB7
:1010C00071EF88F0D7C076F0D8C077F071EF88F074
:1010D000D8BF6DEF88F06FEF88F05CEF88F062EFBB
:1010E00088F0670E7B19D8A478EF88F07AEF88F043
:1010F000A9EF88F08BAF88EF88F0FC0E8A5DFF0EB9
:101100008B59D8A086EF88F088EF88F0A7EF88F099
:10111000FF0E466EFF0E476E76C048F077C049F06E
:1011200046504826475049228A51485C4950800A17
:101130004A6E8B51800A4A58D8A0A1EF88F0A3EFDD
:1011400088F0A7EF88F0660E7A6FA9EF88F0650E39
:101150007A6F76C06CF077C06DF0670E7B19D8A4FB
:10116000B4EF88F0B6EF88F0C6EF88F0660E7A1913
:10117000D8A4BDEF88F0BFEF88F0C8EF88F08BBF30
:10118000C6EF88F0C4EF88F0C8EF88F06C4B6D2B89
:10119000660E7A19D8A4CFEF88F0D1EF88F0F1EF7E
:1011A00088F08BBFD8EF88F0D6EF88F0E4EF88F0B6
:1011B000000E8E6F000E8F6F800E906F3F0E916F3E
:1011C000000E8B6F000E8A6F670E7B19D8B4EBEFA1
:1011D00088F0EDEF88F0F1EF88F08A516C278B51A1
:1011E0006D23000E856F000E846F86C07CF087C073
:1011F0007DF088C07EF089C07FF08EC06EF08FC019
:101200006FF090C070F091C071F082EF89F07CC0F7
:1012100012F07DC013F07EC014F07FC015F08EC0B8
:1012200016F08FC017F090C018F091C019F0F2ECD2
:1012300096F012C02BF013C02CF014C02DF015C086
:101240002EF0BEEC9CF02BC080F02CC081F02DC0A5
:1012500082F02EC083F080C004F081C005F082C00F
:1012600006F083C007F022ECA5F004C072F005C0C0
:1012700073F07CC01DF07DC01EF07EC01FF07FC0EB
:1012800020F08EC008F08FC009F090C00AF091C025
:101290000BF080C004F081C005F082C006F083C06E
:1012A00007F0CBEC94F004C021F005C022F006C09A
:1012B00023F007C024F011ECB2F01DC07CF01EC07A
:1012C0007DF01FC07EF020C07FF08EC012F08FC076
:1012D00013F090C014F091C015F0000E166E000EC1
:1012E000176E200E186E410E196EF2EC96F012C0B9
:1012F0008EF013C08FF014C090F015C091F0000173
:10130000844B852B6C51845D8551800A466E6D51EE
:10131000800A4658D8A08FEF89F091EF89F007EF47
:1013200089F08EC004F08FC005F090C006F091C027
:1013300007F0000E086E000E096EA00E0A6E400E39
:101340000B6ECBEC94F004C080F005C081F006C0B9
:1013500082F007C083F07CC01DF07DC01EF07EC00F
:101360001FF07FC020F080C021F081C022F082C039
:1013700023F083C024F0A5ECA5F0D8B0C2EF89F02B
:10138000C4EF89F0CFEF89F0000E0001806F000EEE
:10139000816F000E826F000E836FF8EF89F07CC0C2
:1013A00004F07DC005F07EC006F07FC007F080C06D
:1013B00008F081C009F082C00AF083C00BF043EC52
:1013C000AAF0D8A0E6EF89F0E8EF89F0F8EF89F00D
:1013D000000172B1EEEF89F0F0EF89F0F8EF89F0DB
:1013E000000E806F000E816F000E826F000E836F03
:1013F00086C004F087C005F088C006F089C007F0F9
:1014000080C008F081C009F082C00AF083C00BF0F0
:101410006BEC92F004C07CF005C07DF006C07EF05D
:1014200007C07FF07CC01DF07DC01EF07EC01FF0A5
:101430007FC020F0000E086E000E096E200E0A6EAE
:10144000410E0B6E6EC004F06FC005F070C006F068
:1014500071C007F0CBEC94F004C021F005C022F07D
:1014600006C023F007C024F0A5ECA5F0D8A03BEF00
:101470008AF03DEF8AF066EF8AF000018A4B8B2BF1
:101480006EC004F06FC005F070C006F071C007F0C8
:10149000000E086E000E096E200E0A6E410E0B6ED5
:1014A000CBEC94F004C06EF005C06FF006C070F095
:1014B00007C071F0660E00017A19D8A462EF8AF0B5
:1014C00064EF8AF066EF8AF06C4B6D2B6EC08EF085
:1014D0006FC08FF070C090F071C091F0650E000188
:1014E0007A19D8B476EF8AF078EF8AF07EEF8AF036
:1014F0008AC06AF08BC06BF082EF8AF0000E6B6FCF
:10150000000E6A6F000E696F000E686F000E676F45
:10151000000E666F000E856F000E846F7DEF8BF0FE
:101520007CC012F07DC013F07EC014F07FC015F0B7
:101530008EC016F08FC017F090C018F091C019F04F
:10154000F2EC96F012C02BF013C02CF014C02DF06A
:1015500015C02EF0BEEC9CF02BC080F02CC081F0AA
:101560002DC082F02EC083F080C004F081C005F051
:1015700082C006F083C007F022ECA5F004C072F030
:1015800005C073F00001D9B9C8EF8AF0CAEF8AF03C
:10159000E7EF8AF072517311D8A4D1EF8AF0D3EF3C
:1015A0008AF0E7EF8AF0670E7B19D8A4DAEF8AF0A9
:1015B000DCEF8AF0E7EF8AF06BBFE3EF8AF0E1EF50
:1015C0008AF0E7EF8AF0664B672B31EF8BF06851BA
:1015D0006911D8A4EEEF8AF0F0EF8AF01AEF8BF0E1
:1015E0006BBFF7EF8AF0F5EF8AF01AEF8BF0800E01
:1015F0008C25D96E010E8D21DA6E2E0EDF6E8C4B8E
:101600008D2B7807D8A07907000E696F010E686FDF
:101610001AEF8BF0800E8C25D96E010E8D21DA6EBB
:10162000300EDF6E8C4B8D2B7807D8A079076607BC
:10163000D8A0670766516711D8A421EF8BF023EF7C
:101640008BF00AEF8BF0800E8C25D96E010E8D2168
:10165000DA6E7251300FDF6E8C4B8D2B7807D8A06D
:1016600079077CC01DF07DC01EF07EC01FF07FC0DA
:1016700020F08EC008F08FC009F090C00AF091C031
:101680000BF080C004F081C005F082C006F083C07A
:1016900007F0CBEC94F004C021F005C022F006C0A6
:1016A00023F007C024F011ECB2F01DC07CF01EC086
:1016B0007DF01FC07EF020C07FF08EC012F08FC082
:1016C00013F090C014F091C015F0000E166E000ECD
:1016D000176E200E186E410E196EF2EC96F012C0C5
:1016E0008EF013C08FF014C090F015C091F000017F
:1016F0006A07D8A06B07844B852B6C51845D85519C
:10170000800A466E6D51800A4658D8B08AEF8BF039
:101710008CEF8BF09AEF8BF08DBF98EF8BF08D51A3
:1017200009E14B0E8C5DD8A098EF8BF09AEF8BF00F
:1017300090EF8AF068516911D8A4A1EF8BF0A3EF64
:101740008BF0B4EF8BF0D9A9A8EF8BF0AAEF8BF058
:10175000B4EF8BF0800E8C25D96E010E8D21DA6EE0
:101760002E0EDF6E8C4B8D2B800E8C25D96E010ECC
:101770008D21DA6E000EDF6E650E7A19D8A4C3EFE4
:101780008BF0C5EF8BF02BEF87F0000E856F4F0EBF
:10179000846F800E8425D96E010E8521DA6E000ECD
:1017A000DF6E000E756F000E746F8BBFDCEF8BF079
:1017B000DAEF8BF0E4EF8BF0000E756F010E746FB3
:1017C0008A6D8B1FD8B08B2B000E776F020E766F51
:1017D00015EF8CF08407D8A08507800E8425D96E7C
:1017E000010E8521DA6E8AC004F08BC005F0000E70
:1017F000076E0A0E066EEBECA9F00450300FDF6E98
:101800008AC004F08BC005F0000E076E0A0E066E4B
:101810002DECA9F004C08AF005C08BF0000176071A
:10182000D8A077077807D8A079078A518B11D8A458
:101830001CEF8CF01EEF8CF0EAEF8BF077BF2BEFF4
:101840008CF0775106E17605D8B029EF8CF02BEFBC
:101850008CF0EAEF8BF08407D8A0850774517511DE
:10186000D8A435EF8CF037EF8CF03DEF8CF0000E04
:10187000636F2B0E626F41EF8CF0000E636F2D0EC5
:10188000626F800E8425D96E010E8521DA6E6000AC
:101890008BF1DFFF7807D8A079078407D8A08507E8
:1018A000BF0E466EFF0E476E4550486E496A465061
:1018B000482647504922495009E11A0E485CD8A0F1
:1018C00064EF8CF066EF8CF06CEF8CF0000E656FBF
:1018D000650E646F70EF8CF0000E656F450E646FDF
:1018E000800E8425D96E010E8521DA6E600093F199
:1018F000DFFF7807D8A07907800E8C25086E010ECF
:101900008D21096E800E84250A6E010E85210B6ED5
:1019100088ECAFF02BEF87F01200600037F1D9FFB1
:1019200060003BF1DAFF6F007BFFF6FF6F0077FF8F
:10193000F7FF000EF86E0800F550250AD8A4A3EFB3
:101940008CF0A5EF8CF047EF92F0600037F1D9FFF3
:1019500060003BF1DAFFDE2A000EDD22000E0001FE
:10196000D66F000ED56FD5C0D9F0D6C0DAF0D769E2
:10197000D869000E9D6F000E9C6F0DEF8DF0D98120
:10198000600037F1D9FF60003BF1DAFFDE2A000E7C
:10199000DD220DEF8DF0D983C0EF8CF0D985C0EF3B
:1019A0008CF0D987C0EF8CF0D989C0EF8CF0000E95
:1019B0009D6F010E9C6F0DEF8DF0600037F1D9FF28
:1019C00060003BF1DAFF6F007BFFF6FF6F0077FFEF
:1019D000F7FF000EF86E0800F550516E526A525033
:1019E000000AD8B4F6EF8CF0D7EF8CF05150200AF3
:1019F000D8B4D1EF8CF0030AD8B4D4EF8CF0080A35
:101A0000D8B4CEEF8CF0060AD8B4BFEF8CF01D0A24
:101A1000D8B4CBEF8CF0D7EF8CF09C519D11D8B49B
:101A200014EF8DF016EF8DF0DDEF8CF0D9A11BEFE8
:101A30008DF01DEF8DF01EEF8DF0D993600037F122
:101A4000D9FF60003BF1DAFF6F007BFFF6FF6F000C
:101A500077FFF7FF000EF86E0800F5502A0AD8A4A9
:101A600034EF8DF036EF8DF069EF8DF0600037F1D7
:101A7000D9FF60003BF1DAFFDE2A000EDD226000B4
:101A80003FF1D9FF600043F1DAFF6F007CFF51F0B6
:101A9000020EDE266F007CFF52F0000EDD22600099
:101AA00047F1D9FF60004BF1DAFF6F0078FFD5F006
:101AB0006F0074FFD6F0D6BF62EF8DF060EF8DF04F
:101AC000ABEF8DF0D981D56DD61FD8B0D62BABEF4B
:101AD0008DF0600037F1D9FF60003BF1DAFF6F0055
:101AE00078FF0BF06F0074FF0CF03BECA1F00BC023
:101AF000D5F00CC0D6F086EF8DF0600037F1D9FF3D
:101B000060003BF1DAFFDE2A000EDD22D00E516EBE
:101B1000FF0E526E600037F1D9FF60003BF1DAFF33
:101B20006F007BFFF6FF6F0077FFF7FF000EF86E88
:101B30000800F550536E546A5150532652505422A7
:101B4000545009E10A0E535CD8A0A9EF8DF0ABEF19
:101B50008DF07DEF8DF0600037F1D9FF60003BF133
:101B6000DAFF6F007BFFF6FF6F0077FFF7FF000ED5
:101B7000F86E0800F5502E0AD8A4C1EF8DF0C3EF1F
:101B80008DF052EF8EF0000E0001D86F000ED76F6F
:101B9000600037F1D9FF60003BF1DAFFDE2A000E6A
:101BA000DD22600037F1D9FF60003BF1DAFF6F0002
:101BB0007BFFF6FF6F0077FFF7FF000EF86E08005F
:101BC000F5502A0AD8A4E7EF8DF0E9EF8DF010EF79
:101BD0008EF0600037F1D9FF60003BF1DAFFDE2ABA
:101BE000000EDD2260003FF1D9FF600043F1DAFF13
:101BF0006F007CFF51F0020EDE266F007CFF52F07A
:101C0000000EDD22600047F1D9FF60004BF1DAFFE2
:101C10006F0078FFD7F06F0074FFD8F052EF8EF0AE
:101C2000600037F1D9FF60003BF1DAFF6F0078FF09
:101C30000BF06F0074FF0CF03BECA1F00BC0D7F081
:101C40000CC0D8F02DEF8EF0600037F1D9FF6000A6
:101C50003BF1DAFFDE2A000EDD22D00E516EFF0EC0
:101C6000526E600037F1D9FF60003BF1DAFF6F0080
:101C70007BFFF6FF6F0077FFF7FF000EF86E08009E
:101C8000F550536E546A51505326525054225450BA
:101C900009E10A0E535CD8A050EF8EF052EF8EF09F
:101CA00024EF8EF0600037F1D9FF60003BF1DAFFDE
:101CB0006F007BFFF6FF6F0077FFF7FF000EF86EF7
:101CC0000800F5500A6E0B6AEEECB1F00A50000104
:101CD000AC6FAC51D8B46FEF8EF071EF8EF0BBEFFC
:101CE0008EF0600037F1D9FF60003BF1DAFF6F0042
:101CF00078FF51F06F0074FF52F0010E5126000E74
:101D00005222600047F1F6FF60004BF1F7FF000E32
:101D1000F86E0800F5500A6E0B6AEEECB1F00A504E
:101D20000001AD6FAD51D8B498EF8EF09AEF8EF000
:101D3000BBEF8EF0600037F1D9FF60003BF1DAFFB6
:101D40006F0078FF51F06F0074FF52F0020E5126C1
:101D5000000E5222600047F1F6FF60004BF1F7FFE2
:101D6000000EF86E0800F5500A6E0B6AEEECB1F04A
:101D70000A500001AE6F600037F1D9FF60003BF1FF
:101D8000DAFF6F007BFFF6FF6F0077FFF7FF000EB3
:101D9000F86E0800F550630AD8A4D1EF8EF0D3EFA7
:101DA0008EF002EF8FF0600037F1D9FF60003BF159
:101DB000DAFFDE2A000EDD2260003FF1D9FF60006D
:101DC00043F1DAFF6F007CFF51F0020EDE266F0058
:101DD0007CFF52F0000EDD22600047F1D9FF600069
:101DE0004BF1DAFFDF50AF6F4BC00DF04CC00EF07F
:101DF000AFC00FF01EECA7F00DC04BF00EC04CF0C2
:101E00006AEF92F0600037F1D9FF60003BF1DAFF32
:101E10006F007BFFF6FF6F0077FFF7FF000EF86E95
:101E20000800F550640AD8B418EF8FF01AEF8FF05D
:101E300032EF8FF0600037F1D9FF60003BF1DAFF3D
:101E40006F007BFFF6FF6F0077FFF7FF000EF86E65
:101E50000800F550690AD8A430EF8FF032EF8FF008
:101E60007CEF8FF0600037F1D9FF60003BF1DAFFC3
:101E7000DE2A000EDD2260003FF1D9FF600043F151
:101E8000DAFF6F007CFF51F0020EDE266F007CFF50
:101E900052F0000EDD22600047F1D9FF60004BF1E7
:101EA000DAFF6F0078FF92F06F0074FF93F0000E7E
:101EB00093BFFF0E946F956F966F976F986F996FA2
:101EC0004BC01FF04CC020F092C021F093C022F014
:101ED00094C023F095C024F096C025F097C026F05A
:101EE00098C027F099C028F0BFEC98F01FC04BF0C5
:101EF00020C04CF06AEF92F0660EAC19D8A483EFC4
:101F00008FF085EF8FF0D8EF8FF0600037F1D9FFB9
:101F100060003BF1DAFF6F007BFFF6FF6F0077FF99
:101F2000F7FF000EF86E08006F00D4FFAFF06000FE
:101F300037F1D9FF60003BF1DAFFDE2A000EDD2227
:101F400060003FF1D9FF600043F1DAFF6F007CFFD2
:101F500051F0040EDE266F007CFF52F0000EDD22F1
:101F6000600047F1D9FF60004BF1DAFF6F0078FFA6
:101F7000A8F06F0078FFA9F06F0078FFAAF06F005B
:101F800078FFABF04BC03FF04CC040F0A8C041F030
:101F9000A9C042F0AAC043F0ABC044F0AFC045F0C6
:101FA00084EC86F03FC04BF040C04CF06AEF92F0FA
:101FB000AC0E046E000E056EFB0E066EFF0E076E75
:101FC000000E096E020E086EACECA2F00450051073
:101FD000D8A4EDEF8FF0EFEF8FF082EF90F060007C
:101FE00037F1D9FF60003BF1DAFF6F0078FF51F065
:101FF0006F0074FF52F0010E5126000E5222600055
:1020000047F1F6FF60004BF1F7FF000EF86E080095
:102010006F00D4FFAFF0BF0E516EFF0E526E600026
:1020200037F1D9FF60003BF1DAFF6F007BFFF6FF6D
:102030006F0077FFF7FF000EF86E0800F550536E43
:10204000546A5150532652505422545007E11A0EEC
:10205000535CD8B02EEF90F030EF90F054EF90F04A
:1020600060003FF1D9FF600043F1DAFF6F007CFFB1
:1020700051F0040EDE266F007CFF52F0000EDD22D0
:10208000600047F1D9FF60004BF1DAFF6F0078FF85
:10209000A8F06F0078FFA9F06F0078FFAAF06F003A
:1020A00078FFABF076EF90F060003FF1D9FF600071
:1020B00043F1DAFF6F007CFF51F0040EDE266F0063
:1020C0007CFF52F0000EDD22600047F1D9FF600076
:1020D0004BF1DAFF6F0078FFA8F06F0078FFA9F0EE
:1020E0006F0078FFAAF06F0078FFABF0020E60007F
:1020F00037F1D9FF60003BF1DAFFDE26000EDD226A
:10210000C2EF8FF0600037F1D9FF60003BF1DAFFDA
:102110006F007BFFF6FF6F0077FFF7FF000EF86E92
:102120000800F550730AD8B498EF90F09AEF90F049
:10213000B9EF90F0600037F1D9FF60003BF1DAFFB2
:102140006F0078FF04F06F0074FF05F0F30E066E69
:10215000FF0E076E000E096E030E086EACECA2F0C7
:1021600004500510D8A4B7EF90F0B9EF90F013EF3A
:1021700091F0600037F1D9FF60003BF1DAFF6F00AA
:102180007BFFF6FF6F0077FFF7FF000EF86E080089
:10219000F550730AD8B4CFEF90F0D1EF90F0D8EFAC
:1021A00090F0000E00019F6F030E9E6FDDEF90F028
:1021B000000E00019F6F010E9E6F600037F1D9FF86
:1021C00060003BF1DAFF9E51DE269F51DD22600068
:1021D0003FF1D9FF600043F1DAFF6F007CFF51F05F
:1021E000020EDE266F007CFF52F0000EDD22600042
:1021F00047F1D9FF60004BF1DAFF6F0078FF9AF0EA
:102200006F0074FF9BF04BC00DF04CC00EF09AC0F5
:102210000FF09BC010F0A3EC9FF00DC04BF00EC070
:102220004CF06AEF92F0600037F1D9FF60003BF1AB
:10223000DAFF6F007BFFF6FF6F0077FFF7FF000EFE
:10224000F86E0800F550750AD8A429EF91F02BEF2D
:1022500091F077EF91F0600037F1D9FF60003BF12A
:10226000DAFFDE2A000EDD2260003FF1D9FF6000B8
:1022700043F1DAFF6F007CFF51F0020EDE266F00A3
:102280007CFF52F0000EDD22600047F1D9FF6000B4
:102290004BF1DAFF6F0078FF53F06F0074FF54F0DA
:1022A00053C0A0F054C0A1F00001A26BA36BA46BBB
:1022B000A56BA66BA76B4BC01FF04CC020F0A0C055
:1022C00021F0A1C022F0A2C023F0A3C024F0A4C03A
:1022D00025F0A5C026F0A6C027F0A7C028F0C7ECBF
:1022E0009DF01FC04BF020C04CF06AEF92F06000F0
:1022F00037F1D9FF60003BF1DAFF6F007BFFF6FF9B
:102300006F0077FFF7FF000EF86E0800F550780AAF
:10231000D8B48DEF91F08FEF91F0A7EF91F06000BE
:1023200037F1D9FF60003BF1DAFF6F007BFFF6FF6A
:102330006F0077FFF7FF000EF86E0800F550580A9F
:10234000D8A4A5EF91F0A7EF91F007EF92F060000D
:1023500037F1D9FF60003BF1DAFF6F007BFFF6FF3A
:102360006F0077FFF7FF000EF86E08006F00D4FFD4
:10237000AFF0600037F1D9FF60003BF1DAFFDE2AF1
:10238000000EDD2260003FF1D9FF600043F1DAFF6B
:102390006F007CFF51F0020EDE266F007CFF52F0D2
:1023A000000EDD22600047F1D9FF60004BF1DAFF3B
:1023B0006F0078FF53F06F0074FF54F053C0A0F02B
:1023C00054C0A1F00001A26BA36BA46BA56BA66B1C
:1023D000A76B4BC01FF04CC020F0A0C021F0A1C0E3
:1023E00022F0A2C023F0A3C024F0A4C025F0A5C011
:1023F00026F0A6C027F0A7C028F0AFC029F032EC25
:102400009AF01FC04BF020C04CF06AEF92F06000D1
:1024100037F1D9FF60003BF1DAFF6F007BFFF6FF79
:102420006F0077FFF7FF000EF86E0800F550250AE1
:10243000D8A41DEF92F01FEF92F038EF92F06000F9
:1024400037F1D9FF60003BF1DAFFDE2A000EDD2212
:10245000000E056E250E046E4BC006F04CC007F052
:102460008AECA7F0000E4C6E010E4B6E6AEF92F0F4
:10247000600037F1D9FF60003BF1DAFFDE2A000E81
:10248000DD22000E4C6E000E4B6E6AEF92F0600083
:1024900037F1D9FF60003BF1DAFF6F007BFFF6FFF9
:1024A0006F0077FFF7FF000EF86E0800F550046E1E
:1024B000056A4BC006F04CC007F08AECA7F060003C
:1024C00037F1D9FF60003BF1DAFFDE2A000EDD2292
:1024D00032EF92F012000750800B106E0750072465
:1024E000126E06AE76EF92F078EF92F079EF92F0FE
:1024F00012801250D8B47FEF92F081EF92F096EFF5
:1025000092F01228D8A487EF92F089EF92F091EF21
:1025100092F0000E046E000E056E000E066E000EA8
:10252000076E068E000E076E9EEF92F0000E046E90
:10253000000E056E000E066E000E076E0B50800B2F
:10254000116E10501118D8B4A8EF92F0AAEF92F0C3
:10255000ABEF92F0108C0B500B24116E0AAEB3EF60
:1025600092F0B5EF92F0B6EF92F011801150D8B41E
:10257000BCEF92F0BEEF92F0D3EF92F01128D8A406
:10258000C4EF92F0C6EF92F0CEEF92F0000E086E1C
:10259000000E096E000E0A6E000E0B6E0A8E000E03
:1025A0000B6EDBEF92F0000E086E000E096E000E4F
:1025B0000A6E000E0B6E1250115CD8B0E2EF92F072
:1025C000E4EF92F00BEF93F010ACE9EF92F0EBEF49
:1025D00092F0EDEF92F0800E101A12C013F011C0BD
:1025E00012F013C011F004C013F008C004F013C0BF
:1025F00008F005C013F009C005F013C009F006C0CB
:1026000013F00AC006F013C00AF007C013F00BC0A5
:1026100007F013C00BF0000E136E125011C00CF037
:102620000D6A0C5E000E0D5A0DBE20EF93F00D509A
:1026300009E11A0E0C5CD8A020EF93F022EF93F082
:1026400059EF93F00450051006100710D8A42BEF93
:1026500093F02EEF93F0010E2FEF93F0000E136E18
:10266000000E046E000E056E000E066E000E076E64
:1026700011C012F062EF93F013A041EF93F043EF1B
:1026800093F049EF93F0D89013300109136E4BEF9C
:1026900093F0D890133204A050EF93F052EF93F0E0
:1026A00053EF93F0138E07340732063205320432AB
:1026B000122A1150125CD8A060EF93F062EF93F0F1
:1026C0003CEF93F010BC67EF93F069EF93F0A9EF44
:1026D00093F01250D8A46FEF93F071EF93F07BEF6B
:1026E00093F0000E046E000E056E000E066E000ED6
:1026F000076ECAEF94F008500426095005220A50CC
:1027000006220B50072207A088EF93F08AEF93F080
:1027100036EF94F013A08FEF93F091EF93F097EFD3
:1027200093F0D89013300109136E99EF93F0D8907D
:10273000133204A09EEF93F0A0EF93F0A1EF93F07B
:10274000138E07340732063205320432122A36EF6E
:1027500094F00850045C095005580A500658075078
:10276000800A0C6E0B50800A0C58D8B0BAEF93F068
:10277000BCEF93F0E7EF93F00450085C0C6E05504B
:1027800009580D6E06500A580E6E07500B580F6E02
:10279000FF0E0C24046EFF0E0D20056EFF0E0E20A2
:1027A000066EFF0E0F20076E800E101A136C13506A
:1027B000D8A4DDEF93F0DFEF93F0EFEF93F0010E8D
:1027C0000426000E052206220722EFEF93F00850A0
:1027D000045E0950055A0A50065A0B50075A045015
:1027E000051006100710D8A4F8EF93F0FAEF93F055
:1027F0002FEF94F01350D8A400EF94F002EF94F070
:102800002FEF94F0000E046E000E056E000E066EA3
:10281000000E076ECAEF94F0D890043605360636DF
:10282000073613AE16EF94F018EF94F019EF94F00A
:10283000048013A01EEF94F020EF94F024EF94F0A6
:10284000D880133626EF94F0D89013361250D8B4AF
:102850002CEF94F02EEF94F02FEF94F0120606AECA
:1028600034EF94F036EF94F00CEF94F0000E116E0C
:1028700013AE3DEF94F03FEF94F057EF94F013C098
:102880000CF07F0E0C16D8B448EF94F04AEF94F099
:102890004EEF94F0010E116E57EF94F004A053EF39
:1028A00094F055EF94F057EF94F04AEF94F01150F4
:1028B000D8B45DEF94F05FEF94F08AEF94F0010EDE
:1028C0000426000E05220622072207A06AEF94F0D4
:1028D0006CEF94F08AEF94F004C00CF005C00DF09A
:1028E00006C00EF007C00FF00F340F320E320D325B
:1028F0000C320CC004F00DC005F00EC006F00FC085
:1029000007F01228D8B487EF94F089EF94F08AEF9B
:1029100094F0122A1228D8B490EF94F092EF94F029
:102920009AEF94F01250D8A498EF94F09AEF94F0A4
:10293000ACEF94F0000E046E000E056E000E066EF5
:10294000000E076E1250D8A4A8EF94F0AAEF94F0EE
:10295000ACEF94F0000E106E12A0B1EF94F0B3EF54
:1029600094F0B6EF94F0068EB7EF94F0069ED890F0
:102970001230076E10AEBFEF94F0C1EF94F0C2EFCB
:1029800094F0078E04C004F005C005F006C006F000
:1029900007C007F012000750800B106E0750072485
:1029A000166E06AED6EF94F0D8EF94F0D9EF94F00F
:1029B00016801650D8B4DFEF94F0E1EF94F0F4EF06
:1029C00094F01628D8A4E7EF94F0E9EF94F0F1EF33
:1029D00094F0000E046E000E056E000E066E000EE2
:1029E000076E068EFCEF94F0000E046E000E056E6E
:1029F000000E066E000E076E0B50800B101A0B5067
:102A00000B24116E0AAE07EF95F009EF95F00AEF6F
:102A100095F011801150D8B410EF95F012EF95F0A9
:102A200025EF95F01128D8A418EF95F01AEF95F03E
:102A300022EF95F0000E086E000E096E000E0A6E71
:102A4000000E0B6E0A8E2DEF95F0000E086E000E34
:102A5000096E000E0A6E000E0B6E1150D8B433EFE3
:102A600095F035EF95F03DEF95F01650D8A43BEF7B
:102A700095F03DEF95F047EF95F0000E046E000ED7
:102A8000056E000E066E000E076EF1EF96F00A500E
:102A900004026F00CCFF1BF06F00D0FF1CF01B5036
:102AA000126E136A146A156A1C50176E186A196A36
:102AB0001A6A095005026F00CCFF1BF06F00D0FFAF
:102AC0001CF01B501226000E1322142215221C503B
:102AD0001726000E182219221A22085006026F002B
:102AE000CCFF1BF06F00D0FF1CF01B501226000E15
:102AF0001322142215221C501726000E1822192208
:102B00001A2214C015F013C014F012C013F0126A88
:102B1000085005026F00CCFF1BF06F00D0FF1CF0C7
:102B20001B5012261C501322000E1422000E1522D8
:102B3000095004026F00CCFF1BF06F00D0FF1CF0A7
:102B40001B5012261C501322000E1422000E1522B8
:102B500014C015F013C014F012C013F0126A08501C
:102B600004026F00CCFF1BF06F00D0FF1CF01B5065
:102B700012261C501322000E1422000E15220A5099
:102B800005026F00CCFF1BF06F00D0FF1CF01B5044
:102B900017261C501822000E1922000E1A22095066
:102BA00006026F00CCFF1BF06F00D0FF1CF01B5023
:102BB00017261C501822000E1922000E1A220A5045
:102BC00006026F00CCFF1BF06F00D0FF1CF01B5003
:102BD0000C6E1C500D6E0E6A0F6A0EC00FF00DC009
:102BE0000EF00CC00DF00C6A0C5017260D50182278
:102BF0000E5019220F501A2212C00CF013C00DF003
:102C000014C00EF015C00FF0190E0CEF96F0D8900E
:102C10000F320E320D320C32E82E07EF96F00C50C8
:102C200017260D5018220E5019220F501A2214C0C8
:102C300015F013C014F012C013F0126A115016C030
:102C40000CF00D6A0C26000E0D22820E0C241B6E59
:102C5000FF0E0D201C6E42EF96F0D89017361836F6
:102C600019361A3615AE37EF96F039EF96F03AEF7F
:102C700096F01780D89012361336143615361B0688
:102C8000D8A01C0619AE47EF96F049EF96F02DEF4D
:102C900096F0000E116E15AE50EF96F052EF96F0D2
:102CA00076EF96F0FF0E12140C6EFF0E13140D6EDD
:102CB000FF0E14140E6E7F0E15140F6E0C500D10B7
:102CC0000E100F10D8B467EF96F069EF96F06DEF25
:102CD00096F0010E116E76EF96F017A072EF96F057
:102CE00074EF96F076EF96F069EF96F01150D8B445
:102CF0007CEF96F07EEF96F0A2EF96F0010E17268D
:102D0000000E182219221A221AA089EF96F08BEFD2
:102D100096F0A2EF96F017C00CF018C00DF019C095
:102D20000EF01AC00FF00F340F320E320D320C328B
:102D30000CC017F00DC018F00EC019F00FC01AF03B
:102D40001B4A1C2A1CBEADEF96F01C5008E11B2844
:102D5000D8A0ADEF96F0AFEF96F0B9EF96F0000E79
:102D6000176E000E186E800E196E7F0E1A6EE7EF4A
:102D700096F01CBEC6EF96F01C5006E11B04D8B0BE
:102D8000C4EF96F0C6EF96F0D2EF96F0000E176EF5
:102D9000000E186E000E196E000E1A6E000E106EE8
:102DA000E7EF96F01BC016F0FF0E1716FF0E181671
:102DB0007F0E1916000E1A1616A0E1EF96F0E3EF3B
:102DC00096F0E4EF96F0198ED89016301A6E1050E7
:102DD0001A1217C004F018C005F019C006F01AC086
:102DE00007F012001550800B226E15501524296E25
:102DF00014AEFDEF96F0FFEF96F000EF97F029800C
:102E00002950D8B406EF97F008EF97F01DEF97F030
:102E10002928D8A40EEF97F010EF97F018EF97F04D
:102E2000000E126E000E136E000E146E000E156E64
:102E3000148E000E156E25EF97F0000E126E000E28
:102E4000136E000E146E000E156E1950800B221AB0
:102E5000195019242A6E18AE30EF97F032EF97F020
:102E600033EF97F02A802A50D8B439EF97F03BEF30
:102E700097F050EF97F02A28D8A441EF97F043EF4E
:102E800097F04BEF97F0000E166E000E176E000EC7
:102E9000186E000E196E188E000E196E58EF97F00E
:102EA000000E166E000E176E000E186E000E196ED4
:102EB0001650171018101910D8A461EF97F063EF8F
:102EC00097F07BEF97F0000E126E000E136E000E5F
:102ED000146E000E156E800E14127F0E1512225005
:102EE000151212C012F013C013F014C014F015C064
:102EF00015F0BEEF98F02950D8A481EF97F083EF3A
:102F000097F08DEF97F0000E126E000E136E000E0C
:102F1000146E000E156EBEEF98F02A5029C01AF0FC
:102F20001B6A1A5E000E1B5A7F0E1A24236E000EB7
:102F30001B20246E12C01EF013C01FF014C020F01E
:102F400015C021F0000E126E000E136E000E146EEE
:102F5000000E156E000E256E000E266E000E276EFA
:102F6000000E286E000E2A6EEEEF97F02A50D8B4AD
:102F7000BCEF97F0BEEF97F0D5EF97F0D8901E36E4
:102F80001F3620362136D8901236133614361536B1
:102F900028AECDEF97F0CFEF97F0D0EF97F01280FB
:102FA000D890253626362736283616501E5C175000
:102FB0001F581850205819502158D8A0E2EF97F008
:102FC000E4EF97F0EDEF97F0288C16501E5E175047
:102FD0001F5A1850205A1950215A2A2A190E2A64A9
:102FE000F4EF97F0F6EF97F0B6EF97F01E501F1042
:102FF00020102110D8B4FFEF97F001EF98F019EFEF
:1030000098F0258019EF98F0D890123613361436C0
:10301000153628AE0EEF98F010EF98F011EF98F0FB
:103020001280D89025362636273628362306D8A093
:10303000240614AE1EEF98F020EF98F004EF98F0FD
:10304000000E2A6E28AE27EF98F029EF98F04DEF8A
:1030500098F0FF0E25141A6EFF0E26141B6EFF0E3D
:1030600027141C6E7F0E28141D6E1A501B101C1086
:103070001D10D8B43EEF98F040EF98F044EF98F070
:10308000010E2A6E4DEF98F012A049EF98F04BEF29
:1030900098F04DEF98F040EF98F02A50D8B453EFE5
:1030A00098F055EF98F079EF98F0010E1226000E87
:1030B00013221422152215A060EF98F062EF98F009
:1030C00079EF98F012C01AF013C01BF014C01CF076
:1030D00015C01DF01D341D321C321B321A321AC0AD
:1030E00012F01BC013F01CC014F01DC015F0234AD1
:1030F000242A24BE84EF98F0245008E12328D8A085
:1031000084EF98F086EF98F091EF98F0000E246E1F
:103110002368000E126E000E136E000E146E000E69
:10312000156E24BE9EEF98F0245006E12304D8B01B
:103130009CEF98F09EEF98F0ACEF98F0000E246EA4
:10314000000E236E000E126E000E136E000E146E33
:10315000000E156E000E226E23C029F029A0B3EFD9
:1031600098F0B5EF98F0B8EF98F0148EB9EF98F0AA
:10317000149ED8902930156E6FEF97F0120021C081
:1031800039F022C03AF023C03BF024C03CF025C007
:103190003DF026C03EF027C03FF028C040F040BEC2
:1031A000D4EF98F0D7EF98F0010ED8EF98F0000E1A
:1031B000376E386A37503810D8B4E1EF98F0E3EF43
:1031C00098F0F3EF98F0401E3F1E3E1E3D1E3C1E41
:1031D0003B1E3A1E396C000E3A223B223C223D2215
:1031E0003E223F2240220001D8BFF9EF98F0FBEFCA
:1031F00098F0FCEF98F0D993D8BF09EF99F0D85127
:1032000006E1D705D8B007EF99F009EF99F00FEF75
:1032100099F0000E346E010E336E13EF99F0D7C0A3
:1032200033F0D8C034F0D5C035F0D6C036F03750C2
:103230003810D8A41EEF99F020EF99F027EF99F0FD
:10324000D9A525EF99F027EF99F02AEF99F03506E7
:10325000D8A03606000E426E4F0E416E000E0101E0
:10326000CF6FAFEF99F04106D8A04206800E4124FF
:10327000D96E010E4220DA6E39C004F03AC005F072
:103280003BC006F03CC007F03DC008F03EC009F06E
:103290003FC00AF040C00BF00A0E0C6E000E0D6E1F
:1032A000000E0E6E000E0F6E000E106E000E116EF0
:1032B000000E126E000E136EFAECA1F004C029F09D
:1032C00005C02AF006C02BF007C02CF008C02DF076
:1032D00009C02EF00AC02FF00BC030F029C016F044
:1032E0002BC017F0DCECB2F01650300FDF6E330657
:1032F000D8A034063506D8A0360639C004F03AC046
:1033000005F03BC006F03CC007F03DC008F03EC0F1
:1033100009F03FC00AF040C00BF00A0E0C6E000E20
:103320000D6E000E0E6E000E0F6E000E106E000E73
:10333000116E000E126E000E136E77ECA0F004C03A
:1033400039F005C03AF006C03BF007C03CF008C0B9
:103350003DF009C03EF00AC03FF00BC040F042BE55
:10336000BAEF99F0425008E14104D8A0BAEF99F0C1
:10337000BCEF99F0EDEF99F039503A103B103C104A
:103380003D103E103F104010D8A4C9EF99F0CBEF8C
:1033900099F033EF99F034BED8EF99F0345006E14C
:1033A0003304D8B0D6EF99F0D8EF99F033EF99F015
:1033B00036BEE3EF99F0365008E13504D8A0E3EFCC
:1033C00099F0E5EF99F0EDEF99F00001D9B3EBEF4B
:1033D00099F0EDEF99F033EF99F037503810D8A409
:1033E000F4EF99F0F6EF99F0FEEF99F00001D9A50E
:1033F000FCEF99F0FEEF99F01DEF9AF04106D8A08E
:10340000420637503810D8A408EF9AF00AEF9AF025
:1034100010EF9AF0000E326E2B0E316E14EF9AF010
:10342000000E326E2D0E316E800E4124D96E010ECB
:103430004220DA6E6000C7F0DFFF1FC014F020C02A
:1034400015F0800E4124166E010E4220176E35C015
:1034500018F036C019F0CAECA8F014C01FF015C05F
:1034600020F012000001D8BF38EF9AF03AEF9AF03E
:103470003BEF9AF0D993D8BF48EF9AF0D85106E1C4
:10348000D705D8B046EF9AF048EF9AF04EEF9AF091
:10349000000E336E010E326E52EF9AF0D7C032F04A
:1034A000D8C033F0D5C034F0D6C035F0D9A95BEF21
:1034B0009AF05DEF9AF061EF9AF0FE0E3426FF0E5F
:1034C000352221C036F022C037F023C038F024C0A6
:1034D00039F025C03AF026C03BF027C03CF028C0A8
:1034E0003DF0000E3F6E4F0E3E6E000E0101CF6F9D
:1034F00014EF9BF03E06D8A03F060F0E3614406E28
:10350000416A41BE8DEF9AF0415009E10A0E405CDC
:10351000D8A08DEF9AF08FEF9AF097EF9AF0570EB0
:103520004024406E000E4120416E9DEF9AF0300E17
:103530004024406E000E4120416EBF0E2A6EFF0EE9
:103540002B6E29502C6E2D6A2A502C262B502D22A2
:103550002D5007E11A0E2C5CD8B0B1EF9AF0B3EF02
:103560009AF0D6EF9AF09F0E2A6EFF0E2B6E200E69
:1035700040102C6E000E41102D6E2A502C262B5020
:103580002D222D5007E11A0E2C5CD8B0CAEF9AF00C
:10359000CCEF9AF0D6EF9AF040C00AF041C00BF0A1
:1035A00057ECB2F00AC040F00BC041F0800E3E2450
:1035B000D96E010E3F20DA6E600003F1DFFF3206A4
:1035C000D8A033063406D8A0350636C02AF037C056
:1035D0002BF038C02CF039C02DF03AC02EF03BC093
:1035E0002FF03CC030F03DC031F0050E01EF9BF0F4
:1035F000D890313230322F322E322D322C322B32C3
:103600002A32E82EF8EF9AF02AC036F02BC037F0B5
:103610002CC038F02DC039F02EC03AF02FC03BF04E
:1036200030C03CF031C03DF03FBE20EF9BF03F503A
:1036300009E1020E3E5CD8A020EF9BF022EF9BF048
:1036400053EF9BF036503710381039103A103B10BA
:103650003C103D10D8A42FEF9BF031EF9BF07AEF98
:103660009AF033BE3EEF9BF0335006E13204D8B0FF
:103670003CEF9BF03EEF9BF07AEF9AF035BE49EFBE
:103680009BF0355008E13404D8A049EF9BF04BEF94
:103690009BF053EF9BF00001D9B351EF9BF053EF38
:1036A0009BF07AEF9AF00001D9A959EF9BF05BEFFC
:1036B0009BF072EF9BF03E06D8A03F06800E3E24A2
:1036C000D96E010E3F20DA6E6000A7F0DFFF3E06E4
:1036D000D8A03F06800E3E24D96E010E3F20DA6E40
:1036E000300EDF6E1FC014F020C015F0800E3E2497
:1036F000166E010E3F20176E34C018F035C019F059
:10370000CAECA8F014C01FF015C020F01200000E83
:103710000001E16F030EE26F600087F3D9FF6000E4
:103720008BF3DAFF000EDF6E3D017599738F000E8B
:103730000001D26F020ED16FD1C004F0D2C005F0EB
:10374000E2ECB3F00009D8B4A8EF9BF0AAEF9BF02D
:10375000A3EF9CF00001D235D231576ED131596EB2
:1037600057C05AF0E1C0B6F0E2C0B7F0FD0EB86F36
:10377000FC0EB96FD1C0BAF0D2C0BBF059C0BCF0DA
:103780005AC0BDF0FEECB0F049EF9CF0E1C012F081
:10379000E2C013F05C0E146EFE0E156E7EECB5F0FA
:1037A0009BEF9CF0200E046E020E056E690E066EF5
:1037B000FF0E076E72ECAEF0E1C004F0E2C005F05F
:1037C000A7ECB0F004C0CFF005C0D0F00001CF519D
:1037D000E125086ED051E221096E200E0A6E020E1C
:1037E0000B6E88ECAFF09BEF9CF0E1C012F0E2C0F2
:1037F00013F0570E146EFF0E156E7EECB5F09BEFB6
:103800009CF0E1C012F0E2C013F0320E146EFF0E15
:10381000156E7EECB5F09BEF9CF0E1C012F0E2C0BB
:1038200013F0970E146EFF0E156E7EECB5F09BEF45
:103830009CF0E1C012F0E2C013F07A0E146EFF0E9D
:10384000156E7EECB5F09BEF9CF0E1C012F0E2C08B
:1038500013F0C80E146EFF0E156E7EECB5F09BEFE4
:103860009CF0E1C012F0E2C013F0400E146EFE0EA8
:10387000156E7EECB5F09BEF9CF0E1C012F0E2C05B
:1038800013F0A40E146EFF0E156E7EECB5F09BEFD8
:103890009CF059C057F05AC058F05850000AD8B49C
:1038A00054EF9CF03DEF9CF05750200AD8B4C6EF7F
:1038B0009BF0010AD8B4C6EF9BF0030AD8B4C6EF58
:1038C0009BF0010AD8B4C6EF9BF0040AD8B4C6EF47
:1038D0009BF00F0AD8B4D2EF9BF0010AD8B4D2EF14
:1038E0009BF0030AD8B4D2EF9BF01D0AD8B4F5EFD1
:1038F0009BF00F0AD8B401EF9CF0010AD8B401EF95
:103900009CF0030AD8B401EF9CF0010AD8B401EF8F
:103910009CF0070AD8B40DEF9CF06B0AD8B419EFED
:103920009CF03F0AD8B425EF9CF0C80AD8B431EF18
:103930009CF03DEF9CF0E1C004F0E2C005F0E4EC47
:10394000AEF0BBECB4F0020E0001D125D16F000E39
:10395000D221D26FD2BFB6EF9CF0D25109E1FC0E5A
:10396000D15DD8A0B6EF9CF0B8EF9CF09CEF9BF037
:103970003D01739F7589BBECB4F012003CC13BF074
:103980003DC13CF03EC13DF03FC13EF02BC03BF09D
:103990002CC03CF02DC03DF02EC03EF0810E2F6EAD
:1039A000FF0E306E3BC031F03CC032F03DC033F012
:1039B0003EC034F0180EE2EF9CF0D890343233322F
:1039C00032323132E82EDDEF9CF031502F24396E47
:1039D000000E30203A6E3ABEF7EF9CF03A5009E103
:1039E000170E395CD8A0F7EF9CF0F9EF9CF003EFCD
:1039F0009DF02BC02BF02CC02CF02DC02DF02EC034
:103A00002EF0C6EF9DF03ABE08EF9DF00AEF9DF054
:103A10007AEF9DF039C02FF0FF0E306EFF0E316E41
:103A20007F0E326E000E336E2F6619EF9DF021EF80
:103A30009DF0333433323232313230322F2E14EFA4
:103A40009DF030C035F031C036F032C037F033C0B1
:103A500038F035503B142F6E36503C14306E3750D2
:103A60003D14316E38503E14326E2F5030103110EC
:103A70003210D8A43EEF9DF040EF9DF042EF9DF054
:103A8000F9EF9CF03BC02FF03CC030F03DC031F06E
:103A90003EC032F0200E52EF9DF0D89032323132DB
:103AA00030322F32E82E4DEF9DF02F503010311074
:103AB0003210D8B45EEF9DF060EF9DF068EF9DF09E
:103AC00035503B2636503C2237503D2238503E225E
:103AD000351C2F6E361C306E371C316E381C326E22
:103AE0002F503B1630503C1631503D1632503E168A
:103AF000BEEF9DF03BC02FF03CC030F03DC031F038
:103B00003EC032F0200E8AEF9DF0D8903232313232
:103B100030322F32E82E85EF9DF02F5030103110CB
:103B20003210D8A496EF9DF098EF9DF0A2EF9DF093
:103B3000000E3B6E000E3C6E000E3D6E000E3E6EA3
:103B4000BEEF9DF0D8903B342F6E3C34306E3D3448
:103B5000316E3E34326E2F50301031103210D8B4E6
:103B6000B4EF9DF0B6EF9DF0BEEF9DF0000E3B6E02
:103B7000000E3C6E800E3D6EBF0E3E6E3BC02BF0C5
:103B80003CC02CF03DC02DF03EC02EF012000001D4
:103B9000D8BFCDEF9DF0CFEF9DF0D0EF9DF0D99342
:103BA000D8BFDDEF9DF0D85106E1D705D8B0DBEFE7
:103BB0009DF0DDEF9DF0E3EF9DF0000E326E010E03
:103BC000316EE7EF9DF0D7C031F0D8C032F0D5C0EC
:103BD00033F0D6C034F021C035F022C036F023C017
:103BE00037F024C038F025C039F026C03AF027C09D
:103BF0003BF028C03CF0000E3E6E4F0E3D6E000EB6
:103C00000101CF6F7AEF9EF03D06D8A03E06800EF0
:103C10003D24D96E010E3E20DA6E35C004F036C068
:103C200005F037C006F038C007F039C008F03AC0D8
:103C300009F03BC00AF03CC00BF00A0E0C6E000EFF
:103C40000D6E000E0E6E000E0F6E000E106E000E4A
:103C5000116E000E126E000E136E62ECA8F004C01E
:103C600029F005C02AF006C02BF007C02CF008C0D0
:103C70002DF009C02EF00AC02FF00BC030F02950F3
:103C8000300FDF6E3106D8A032063306D8A03406D6
:103C900035C004F036C005F037C006F038C007F074
:103CA00039C008F03AC009F03BC00AF03CC00BF044
:103CB0000A0E0C6E000E0D6E000E0E6E000E0F6ED4
:103CC000000E106E000E116E000E126E000E136EBE
:103CD000A6ECA6F004C035F005C036F006C037F0FB
:103CE00007C038F008C039F009C03AF00AC03BF00C
:103CF0000BC03CF03D503E10D8B481EF9EF083EFF6
:103D00009EF0B4EF9EF03550361037103810391051
:103D10003A103B103C10D8A490EF9EF092EF9EF02A
:103D200004EF9EF032BE9FEF9EF0325006E1310468
:103D3000D8B09DEF9EF09FEF9EF004EF9EF034BE52
:103D4000AAEF9EF0345008E13304D8A0AAEF9EF009
:103D5000ACEF9EF0B4EF9EF00001D9B3B2EF9EF04D
:103D6000B4EF9EF004EF9EF01FC014F020C015F0D9
:103D7000800E3D24166E010E3E20176E33C018F0E3
:103D800034C019F0CAECA8F014C01FF015C020F020
:103D900012000C6E0C50D8B4D0EF9EF0D2EF9EF013
:103DA000F4EF9EF007BED9EF9EF0D7EF9EF0F4EF50
:103DB0009EF004C008F005C009F006C00AF007C074
:103DC0000BF0081E091E0A1E0B1E082A000E0922EF
:103DD0000A220B2208C00EF009C00FF00AC010F032
:103DE0000BC011F0FCEF9EF004C00EF005C00FF008
:103DF00006C010F007C011F004500510061007109F
:103E0000D8A405EF9FF007EF9FF011EF9FF0000E91
:103E1000046E000E056E000E066E000E076EA2EF19
:103E20009FF0960E0D6E1BEF9FF00D2AD890113269
:103E300010320F320E32000E0E14086E000E0F14E8
:103E4000096E000E10140A6EFE0E11140B6E08504F
:103E500009100A100B10D8A430EF9FF032EF9FF03A
:103E600015EF9FF040EF9FF00D2A010E0E26000E79
:103E70000F2210221122D890113210320F320E323E
:103E8000000E0E14086E000E0F14096E000E1014B2
:103E90000A6EFF0E11140B6E085009100A100B1059
:103EA000D8A455EF9FF057EF9FF034EF9FF05FEFEE
:103EB0009FF00D06D8900E360F361036113610BE14
:103EC00064EF9FF066EF9FF06EEF9FF0020E0D60C3
:103ED0006CEF9FF06EEF9FF059EF9FF00DB073EF16
:103EE0009FF075EF9FF076EF9FF0109ED8900D3207
:103EF0000DC008F0096A0A6A0B6A08C00BF00A6A6A
:103F0000096A086A08500E1209500F120A5010125E
:103F10000B5011120C50D8B490EF9FF092EF9FF01D
:103F20009AEF9FF007BE99EF9FF097EF9FF09AEFFF
:103F30009FF0118E0EC004F00FC005F010C006F007
:103F400011C007F0120020EEE8F110EE12F0060E9C
:103F50006F006FFFE3FFE806FBE20FC01DF010C02B
:103F60001EF01D501E10D8A4B8EF9FF0BAEF9FF0BE
:103F7000BEEF9FF0120E1D6E000E1E6E1DC004F0EF
:103F80001EC005F0A7ECB0F004C021F005C022F07F
:103F9000D7C01FF0D8C020F020BED1EF9FF0D3EFE4
:103FA0009FF0E8EF9FF021501F5C2050800A116EB7
:103FB0002250800A1158D8A0E0EF9FF0E2EF9FF066
:103FC000E4EF9FF0E8EF9FF01FC021F020C022F047
:103FD00021C01FF022C020F0D5C01BF0D6C01CF0BD
:103FE0000001D9B1F6EF9FF0F8EF9FF015EFA0F0C8
:103FF00006EFA0F0000E056E200E046E0DC006F058
:104000000EC007F08AECA7F0214A222A1B50215C3F
:104010002250800A116E1C50800A1158D8A013EF4C
:10402000A0F015EFA0F0FAEF9FF0000E1A6E000E50
:10403000196E3EEFA0F0600077F0F6FF60007BF0B5
:10404000F7FF000EF86E1F0EF76403D00800F5505E
:1040500007D06F00DBFFE9FF6F00DFFFEAFFEF50E3
:10406000116E1150046E056A0DC006F00EC007F007
:104070008AECA7F01D4A1E2A194A1A2A1F50195CF9
:104080001A50800A116E2050800A1158D8A04BEFA8
:10409000A0F04DEFA0F01BEFA0F00001D9A153EF6D
:1040A000A0F055EFA0F072EFA0F063EFA0F0000ECB
:1040B000056E200E046E0DC006F00EC007F08AECEF
:1040C000A7F0214A222A1B50215C2250800A116E3F
:1040D0001C50800A1158D8A070EFA0F072EFA0F029
:1040E00057EFA0F021C00DF022C00EF01200000E1C
:1040F000156E13BE80EFA0F07EEFA0F092EFA0F05F
:10410000131E121E111E101E0F1E0E1E0D1E0C6CF5
:10411000000E0D220E220F22102211221222132233
:10412000010E156E0BBE99EFA0F097EFA0F0ABEF6C
:10413000A0F00B1E0A1E091E081E071E061E051EE5
:10414000046C000E052206220722082209220A22F8
:104150000B22010E151A20EE16F0070EDE6AE80695
:10416000FDE20C500D100E100F1010101110121057
:104170001310D8B4BEEFA0F0C0EFA0F012EFA1F082
:10418000010E146ECEEFA0F0D8900C360D360E3620
:104190000F361036113612361336142A13AED3EFFB
:1041A000A0F0D5EFA0F0C4EFA0F0D89016361736E7
:1041B000183619361A361B361C361D360C50045C60
:1041C0000D5005580E5006580F50075810500858FB
:1041D0001150095812500A5813500B58D8A0F3EF39
:1041E000A0F0F5EFA0F006EFA1F00C50045E0D502A
:1041F000055A0E50065A0F50075A1050085A1150BF
:10420000095A12500A5A13500B5A1680D89013327A
:104210001232113210320F320E320D320C32142E95
:10422000D5EFA0F01550D8B418EFA1F01AEFA1F017
:104230002AEFA1F01D1E1C1E1B1E1A1E191E181E81
:10424000171E166C000E1722182219221A221B2282
:104250001C221D2216C004F017C005F018C006F07D
:1042600019C007F01AC008F01BC009F01CC00AF002
:104270001DC00BF01200000E146E000E136E000E27
:10428000126E000E116E47EFA1F00B4A0C2A60006F
:104290002FF0F6FF600033F0F7FF000EF86E080015
:1042A000F550200AD8B457EFA1F059EFA1F045EF2F
:1042B000A1F0F70E0D6EFF0E0E6E60002FF0F6FFF0
:1042C000600033F0F7FF000EF86E0800F5500F6E37
:1042D000106A0D500F260E501022105009E1050EE5
:1042E0000F5CD8A076EFA1F078EFA1F045EFA1F038
:1042F00082EFA1F0000E126E010E116E0B4A0C2A15
:10430000BFEFA1F060002FF0F6FF600033F0F7FF81
:10431000000EF86E0800F5500D6E0E6A0E50000A81
:10432000D8B495EFA1F0BFEFA1F00D502B0AD8B48F
:104330007EEFA1F0060AD8B47AEFA1F0BFEFA1F0AA
:1043400013C004F014C005F0000E076E0A0E066ECE
:104350002CECB5F060002FF0F6FF600033F0F7FFB3
:10436000000EF86E0800F550045E000E055A300E7F
:104370000424136E000E0520146E7EEFA1F0D00E03
:104380000D6EFF0E0E6E60002FF0F6FF600033F032
:10439000F7FF000EF86E0800F5500F6E106A0D5012
:1043A0000F260E501022105009E10A0E0F5CD8A003
:1043B000DCEFA1F0DEEFA1F0A0EFA1F011501210A0
:1043C000D8A4E5EFA1F0E7EFA1F0F5EFA1F013C05D
:1043D0000DF014C00EF00D1E0E1E0D4A0E2A0DC05B
:1043E0000BF00EC00CF0F9EFA1F013C00BF014C0ED
:1043F0000CF01200000E156E0BBE03EFA2F001EFE1
:10440000A2F015EFA2F00B1E0A1E091E081E071EC1
:10441000061E051E046C000E052206220722082235
:1044200009220A220B22010E156E13BE1CEFA2F008
:104430001AEFA2F02CEFA2F0131E121E111E101E76
:104440000F1E0E1E0D1E0C6C000E0D220E220F22D2
:1044500010221122122213220C500D100E100F10D8
:104460001010111012101310D8B439EFA2F03BEF56
:10447000A2F083EFA2F0010E146E49EFA2F0D890E3
:104480000C360D360E360F36103611361236133600
:10449000142A13AE4EEFA2F050EFA2F03FEFA2F0BD
:1044A0000C50045C0D5005580E5006580F5007581C
:1044B000105008581150095812500A5813500B58F0
:1044C000D8A065EFA2F067EFA2F077EFA2F00C5052
:1044D000045E0D50055A0E50065A0F50075A1050E0
:1044E000085A1150095A12500A5A13500B5AD890B0
:1044F00013321232113210320F320E320D320C32B0
:10450000142E50EFA2F01550D8B489EFA2F08BEF23
:10451000A2F09BEFA2F00B1E0A1E091E081E071E2A
:10452000061E051E046C000E052206220722082224
:1045300009220A220B2204C004F005C005F006C0BF
:1045400006F007C007F008C008F009C009F00AC06B
:104550000AF00BC00BF0120004C00BF005C00CF009
:1045600006C00DF007C00EF00806D8A009060828FE
:1045700006E10928D8A4BFEFA2F0C1EFA2F0CEEF68
:10458000A2F0000E056E000E046E54EFA3F00B4A6D
:104590000C2A0D4A0E2A0806D8A0090660002FF042
:1045A000F6FF600033F0F7FF000EF86E1F0EF764A1
:1045B00003D00800F55007D06F00DBFFE9FF6F0064
:1045C000DFFFEAFFEF500009D8B4E9EFA2F0EBEF0C
:1045D000A2F02FEFA3F0600037F0F6FF60003BF091
:1045E000F7FF000EF86E0800F5500009D8B4FBEF95
:1045F000A2F0FDEFA2F02FEFA3F008500910D8B4FD
:1046000004EFA3F006EFA3F02FEFA3F0600037F064
:10461000F6FF60003BF0F7FF000EF86E08006F0039
:10462000D4FF0AF060002FF0F6FF600033F0F7FFD0
:10463000000EF86E1F0EF76403D00800F55007D087
:104640006F00DBFFE9FF6F00DFFFEAFFEF500A18A2
:10465000D8B42DEFA3F02FEFA3F0C7EFA2F06000C6
:104660002FF0F6FF600033F0F7FF000EF86E1F0E1C
:10467000F76403D00800F55007D06F00DBFFE9FFB7
:104680006F00DFFFEAFFEF500A6E600037F0F6FFC1
:1046900060003BF0F7FF000EF86E0800F5500A5C72
:1046A000046E056AD8A005061200400E6FECACF04F
:1046B000030E296E080E286E770EE82EFED7282EE0
:1046C000FCD7292EFAD700F0000E2B6E000E2A6EB2
:1046D00026042710D8A46FEFA3F071EFA3F079EFB1
:1046E000A3F0400E046EF90E056ED3ECB0F0BBECF7
:1046F000B4F0000E2D6E000E2C6E26042710D8A4E8
:1047000084EFA3F086EFA3F0B7EFA3F02C502D10A9
:10471000D8B48DEFA3F08FEFA3F0B7EFA3F0070E9F
:104720002C14286E000E2D14296E28502910D8A4A0
:104730009CEFA3F09EEFA3F0B7EFA3F02AC028F000
:104740002BC029F0D89028362936D890283629361B
:10475000D89028362936400E2824046EF90E2920D8
:10476000056ED3ECB0F02A4A2B2ABBECB4F0010E54
:104770002C24F66EF80E2D20F76EF86A000EF82243
:104780000800F55038ECAEF026042710D8A4CBEF83
:10479000A3F0CDEFA3F0DCEFA3F0010E2C24F66E16
:1047A000F80E2D20F76EF86A000EF8220800F5507A
:1047B00034ECB2F0BBECB4F02C4A2D2A2D5009E1B8
:1047C000400E2C5CD8A0E7EFA3F0E9EFA3F07DEF5B
:1047D000A3F0800E6FECACF0D00E286ECA0EE82E5F
:1047E000FED7282EFCD71200F70E046EFF0E056EC2
:1047F000D3ECB0F0000E226E300E84ECADF0680EFB
:10480000266EE40EE82EFED7262EFCD700D0320E00
:10481000C6ECB5F0000E226E300E84ECADF0150E35
:10482000266EC60EE82EFED7262EFCD700D0330EFD
:10483000C6ECB5F0000E226E300E84ECADF0150E15
:10484000266EC60EE82EFED7262EFCD700D0340EDC
:10485000C6ECB5F0000E226E250E84ECADF0150E00
:10486000266EC60EE82EFED7262EFCD700D0350EBB
:10487000C6ECB5F0010E226E280E84ECADF0150EDC
:10488000266EC60EE82EFED7262EFCD700D0360E9A
:10489000C6ECB5F0010E226E080E84ECADF0150EDC
:1048A000266EC60EE82EFED7262EFCD700D0370E79
:1048B000C6ECB5F0010E226E010E84ECADF0030ED5
:1048C000276E080E266E770EE82EFED7262EFCD712
:1048D000272EFAD700F0380EC6ECB5F0010E226E86
:1048E000060E84ECADF0150E266EC60EE82EFED731
:1048F000262EFCD700D0390EC6ECB5F0010E226E84
:104900000C0E84ECADF0150E266EC60EE82EFED70A
:10491000262EFCD700D0410EC6ECB5F01200A8EC54
:10492000B6F00009D8B497EFA4F099EFA4F0D5EF52
:10493000A4F0A6EFA4F0FDECB6F021EFA5F055EC45
:10494000B7F021EFA5F0000E21EFA5F018C10FF090
:1049500019C110F020EE09F102D8B9EFA4F005005A
:10496000FA6EDE50FD6EDE50FE6EDE50FF6EFA50C7
:104970001200116E126A1250000AD8B4C2EFA4F0ED
:10498000A3EFA4F01150010AD8B4A3EFA4F0030AD6
:10499000D8B49BEFA4F0010AD8B49FEFA4F0070AA3
:1049A000D8B4A3EFA4F0A3EFA4F09DECB6F00009F7
:1049B000D8B4DDEFA4F0DFEFA4F020EFA5F0010103
:1049C0002951030B0009D8B4E8EFA4F0EAEFA4F0F2
:1049D000F6EFA4F0010E116E2951030B126E115067
:1049E000125E29511218FC0B1218296F60008FF407
:1049F000D9FF600093F4DAFFDF50156E234B242BB0
:104A00002507D8A0260725512611D8A40AEFA5F01E
:104A10000CEFA5F014EFA5F045ECADF0116E1150C0
:104A2000136E146A18EFA5F0000E146E030E136EC9
:104A300013C016F0155010ECB7F0165021EFA5F08A
:104A4000030E1200063407340D6E0D50D8A42BEF60
:104A5000A5F02DEFA5F037EFA5F0000E046E000EC7
:104A6000056E000E066E000E076EA4EFA5F004C0E2
:104A700008F005C009F006C00AF007C00BF0200ED0
:104A800047EFA5F0D8900B320A3209320832E82EEF
:104A900042EFA5F008500C6E068EFF0E0416FF0EB6
:104AA0000516FF0E0616000E0716960E0D5E0DBEBD
:104AB0005EEFA5F05CEFA5F074EFA5F00D50800A55
:104AC000970FD8B066EFA5F068EFA5F06AEFA5F0F4
:104AD0002DEFA5F0D89007320632053204320D3E94
:104AE0006AEFA5F08CEFA5F01F0E0D647AEFA5F02C
:104AF0007CEFA5F084EFA5F02DEFA5F0D89004365B
:104B00000536063607360D060D50D8A48AEFA5F0F7
:104B10008CEFA5F07EEFA5F00C50D8B492EFA5F085
:104B200094EFA5F09CEFA5F0071E061E051E046C71
:104B3000000E05220622072204C004F005C005F07D
:104B400006C006F007C007F01200000E1D14256E07
:104B5000000E1E14266E800E1F14276E7F0E20146A
:104B6000286E2550261027102810D8A4BAEFA5F0DB
:104B7000BCEFA5F0C4EFA5F0000E1D6E000E1E6E7A
:104B8000000E1F6E000E206E000E2114256E000E0A
:104B90002214266E800E2314276E7F0E2414286E96
:104BA0002550261027102810D8A4D9EFA5F0DBEF48
:104BB000A5F0E3EFA5F0000E216E000E226E000EB0
:104BC000236E000E246E20AEE8EFA5F0EAEFA5F00C
:104BD000F3EFA5F01D6C1E1ED8B01E2A1F1ED8B004
:104BE0001F2A800E205624AEF8EFA5F0FAEFA5F0AC
:104BF00003EFA6F0216C221ED8B0222A231ED8B0C3
:104C0000232A800E2456000E1D1A000E1E1A000EB6
:104C10001F1A800E201A000E211A000E221A000EF2
:104C2000231A800E241A21501D5C22501E58235036
:104C30001F5824502058D8B020EFA6F022EFA6F03D
:104C400025EFA6F0D89026EFA6F0D880120040C13C
:104C50000EF041C10FF042C110F043C111F004C089
:104C60000EF005C00FF006C010F007C011F00EC026
:104C700008F00FC009F010C00AF011C00BF0180EB8
:104C800047EFA6F0D8900B320A3209320832E82EEC
:104C900042EFA6F008500C6E0D6A0C500D10D8A40F
:104CA00054EFA6F056EFA6F076EFA6F0D8900E34AB
:104CB000086E0F34096E10340A6E11340B6E0850F2
:104CC00009100A100B10D8A468EFA6F06AEFA6F03E
:104CD00070EFA6F0000E056E020E046EA5EFA6F0B2
:104CE000000E056E030E046EA5EFA6F00C280D1045
:104CF000D8A47DEFA6F07FEFA6F0A1EFA6F00EC03E
:104D000008F00FC009F010C00AF011C00BF0090E36
:104D1000D890083609360A360B36E82E88EFA6F00A
:104D2000085009100A100B10D8B499EFA6F09CEFA8
:104D3000A6F0010E9DEFA6F0000E046E056AA5EF29
:104D4000A6F0000E056E040E046E120020EE14F0A4
:104D5000070EDE6AE806FDE20C500D100E100F1073
:104D60001010111012101310D8B4B9EFA6F0BBEF49
:104D7000A6F00DEFA7F0010E1C6EC9EFA6F0D890BB
:104D80000C360D360E360F361036113612361336F7
:104D90001C2A13AECEEFA6F0D0EFA6F0BFEFA6F020
:104DA000D8901436153616361736183619361A3680
:104DB0001B360C50045C0D5005580E5006580F5011
:104DC0000758105008581150095812500A581350DB
:104DD0000B58D8A0EEEFA6F0F0EFA6F001EFA7F089
:104DE0000C50045E0D50055A0E50065A0F50075ACB
:104DF0001050085A1150095A12500A5A13500B5A9F
:104E00001480D89013321232113210320F320E3217
:104E10000D320C321C2ED0EFA6F014C004F015C0D9
:104E200005F016C006F017C007F018C008F019C04A
:104E300009F01AC00AF01BC00BF012000001D55196
:104E4000D611D8A426EFA7F028EFA7F02EEFA7F0F1
:104E5000D5C013F0D6C014F034EFA7F0FF0ED5255F
:104E6000136EFF0ED621146ED9A139EFA7F03BEFD8
:104E7000A7F044EFA7F00FC004F0056A0DC006F0DC
:104E80000EC007F08AECA7F014BE49EFA7F04BEF75
:104E9000A7F04DEFA7F051EFA7F0000E146E000E33
:104EA000136E000E126E000E116E63EFA7F0000E6F
:104EB000056E200E046E0DC006F00EC007F08AECE1
:104EC000A7F0114A122A1350115C1250800A106E7A
:104ED0001450800A1058D8A070EFA7F072EFA7F016
:104EE00057EFA7F00001D9B178EFA7F07AEFA7F05C
:104EF00083EFA7F00FC004F0056A0DC006F00EC0E6
:104F000007F08AECA7F0010E11240D6E000E12209E
:104F10000E6E120006500710D8B491EFA7F093EF71
:104F2000A7F09CEFA7F006500710D8A49AEFA7F0BF
:104F30009CEFA7F0A1EFA7F004505BECB7F0F5EF02
:104F4000A7F020EE09F00650D9260750DA22DE50ED
:104F5000DE10D8B4AEEFA7F0B0EFA7F0CBEFA7F01C
:104F600020EE09F00650D9260750DA2210EE03F0A1
:104F70000650E1260750E222DE50E65CE650800A49
:104F80000C6EDE50800A0C58D8B0C9EFA7F0CBEFFA
:104F9000A7F0F5EFA7F020EE03F00650D926075052
:104FA000DA226F0078FF08F06F0074FF09F06000EC
:104FB0001BF0D9FF60001FF0DAFF6F0078FF0AF0E6
:104FC0006F0074FF0BF008500A24D96E09500B20B3
:104FD000DA6E600013F0DFFF20EE03F00650D926F2
:104FE0000750DA22DE2A000EDD2212002850291096
:104FF000D8A4FDEFA7F0FFEFA7F003EFA8F0000E95
:10500000296E010E286E28500001FA5DFB51800ABE
:105010002B6E2950800A2B58D8B011EFA8F013EF4F
:10502000A8F017EFA8F0FAC028F0FBC029F026047A
:105030002710D8A41EEFA8F020EFA8F024EFA8F0C6
:1050400028507F0F6FECACF0020E26182710D8A462
:105050002CEFA8F02EEFA8F032EFA8F02850BF0FE9
:105060006FECACF0030E26182710D8A43AEFA8F086
:105070003CEFA8F040EFA8F02850930F6FECACF095
:10508000040E26182710D8A448EFA8F04AEFA8F07D
:105090004EEFA8F02850D30F6FECACF0150E2B6E2E
:1050A000C60EE82EFED72B2EFCD700D02A5038ECA7
:1050B000AEF0150E2B6EC60EE82EFED72B2EFCD7AB
:1050C00000D012000C500D100E100F101010111007
:1050D00012101310D8B46FEFA8F071EFA8F0B9EF69
:1050E000A8F0010E146E7FEFA8F0D8900C360D36A4
:1050F0000E360F361036113612361336142A13AE0A
:1051000084EFA8F086EFA8F075EFA8F00C50045CCF
:105110000D5005580E5006580F500758105008589B
:105120001150095812500A5813500B58D8A09BEF31
:10513000A8F09DEFA8F0ADEFA8F00C50045E0D5064
:10514000055A0E50065A0F50075A1050085A11505F
:10515000095A12500A5A13500B5AD890133212326D
:10516000113210320F320E320D320C32142E86EF05
:10517000A8F004C004F005C005F006C006F007C0A2
:1051800007F008C008F009C009F00AC00AF00BC017
:105190000BF012000001D9A1D0EFA8F0D2EFA8F0D7
:1051A000DCEFA8F016C00DF017C00EF014C00FF021
:1051B00015C010F079ECB2F019BEE1EFA8F0E3EF02
:1051C000A8F0E9EFA8F018C01DF019C01EF0EDEF2F
:1051D000A8F0000E1E6E000E1D6E000E1C6E000E5E
:1051E0001B6EFFEFA8F0000E056E200E046E14C0BB
:1051F00006F015C007F08AECA7F01B4A1C2A1D50C8
:105200001B5C1C50800A1A6E1E50800A1A58D8A0C7
:105210000CEFA9F00EEFA9F0F3EFA8F00001D9B15F
:1052200014EFA9F016EFA9F020EFA9F016C00DF0C9
:1052300017C00EF014C00FF015C010F079ECB2F0EA
:1052400016C004F017C005F0A7ECB0F01D50042400
:10525000146E1E500520156E1200000E096E07BE5A
:1052600036EFA9F034EFA9F03CEFA9F0066C071E69
:10527000D8B0072A010E096E05BE43EFA9F041EF31
:10528000A9F049EFA9F0046C051ED8B0052A010E5B
:10529000091A000E0B6E000E0A6E06500710D8B4E5
:1052A00054EFA9F056EFA9F07EEFA9F0010E086EB9
:1052B0005EEFA9F0D89006360736082A07AE63EFEE
:1052C000A9F065EFA9F05AEFA9F0D8900A360B368D
:1052D0000650045C07500558D8A071EFA9F073EF91
:1052E000A9F078EFA9F00650045E0750055A0A802D
:1052F000D89007320632082E65EFA9F00950D8B4CD
:1053000084EFA9F086EFA9F08AEFA9F00A6C0B1ED2
:10531000D8B00B2A0AC004F00BC005F012002A6EA8
:105320002650D8A496EFA9F098EFA9F09AEFA9F02B
:10533000010E266E2650276E286A27500001FA5D5E
:10534000FB51800A296E2850800A2958D8B0ABEF4B
:10535000A9F0ADEFA9F0AFEFA9F0FA05266E2A0487
:10536000D8A4B5EFA9F0B7EFA9F0BBEFA9F026508C
:105370007F0F6FECACF0020E2A18D8A4C2EFA9F090
:10538000C4EFA9F0C8EFA9F02650BF0F6FECACF046
:10539000030E2A18D8A4CFEFA9F0D1EFA9F0D5EFCA
:1053A000A9F02650930F6FECACF0040E2A18D8A485
:1053B000DCEFA9F0DEEFA9F0E2EFA9F02650D30F61
:1053C0006FECACF0150E276EC60EE82EFED7272E1A
:1053D000FCD700D01200000E096E05BEF4EFA9F054
:1053E000F2EFA9F0FAEFA9F0046C051ED8B0052A77
:1053F000010E096E07BE01EFAAF0FFEFA9F005EF5D
:10540000AAF0066C071ED8B0072A06500710D8B4B9
:105410000CEFAAF00EEFAAF032EFAAF0010E086E20
:1054200016EFAAF0D89006360736082A07AE1BEF0B
:10543000AAF01DEFAAF012EFAAF00650045C075084
:105440000558D8A026EFAAF028EFAAF02CEFAAF072
:105450000650045E0750055AD89007320632082ECF
:105460001DEFAAF00950D8B438EFAAF03AEFAAF02D
:105470003EEFAAF0046C051ED8B0052A04C004F063
:1054800005C005F01200000E04140C6E000E051489
:105490000D6E800E06140E6E7F0E07140F6E0C50EC
:1054A0000D100E100F10D8A458EFAAF05AEFAAF062
:1054B00062EFAAF0000E046E000E056E000E066E7E
:1054C000000E076E000E08140C6E000E09140D6E0F
:1054D000800E0A140E6E7F0E0B140F6E0C500D1002
:1054E0000E100F10D8A477EFAAF079EFAAF081EF91
:1054F000AAF0000E086E000E096E000E0A6E000E75
:105500000B6E085004180FE1095005180CE10A5001
:10551000061809E10B500718D8B491EFAAF093EFE1
:10552000AAF096EFAAF0D89097EFAAF0D8801200D0
:10553000046E010E056E010129B7A1EFAAF0A3EFD9
:10554000AAF0E8EFAAF004C022F129952987FC0E01
:1055500029170F0E276F010E216FF40E206F298976
:10556000B20E006F6E0E016F010E026F000E126F11
:10557000000E136FB20E036F6E0E046F010E056FF7
:10558000000E146F000E156FB20E066F6E0E076FD1
:10559000010E086F000E166F000E176FB20E096F26
:1055A0006E0E0A6F010E0B6F000E186F000E196F52
:1055B000AE0E0C6F6E0E0D6F010E0E6F000E1A6F99
:1055C000000E1B6F2FECB7F0D2ECB4F0000E056E9E
:1055D00005501200010129890EEFABF042ECB7F043
:1055E000080E3BEFABF042ECB7F0070E3BEFABF031
:1055F0000101252915ECB7F0040E3BEFABF0070EC7
:1056000001012719D8B407EFABF009EFABF00BEFAE
:10561000ABF045ECB7F00F0E3BEFABF012C10FF063
:1056200013C110F002D81FEFABF00500FA6E005165
:10563000FD6E0151FE6E0251FF6EFA501200116EA6
:10564000126A1250000AD8B428EFABF0FFEFAAF0AC
:105650001150010AD8B4FFEFAAF0030AD8B4F3EF4F
:10566000AAF0010AD8B4EEEFAAF0070AD8B4F8EF0E
:10567000AAF0FFEFAAF01200B3ECB6F00009D8A42C
:1056800044EFABF046EFABF049EFABF0040E8AEF1E
:10569000ABF001012951030B0009D8B452EFABF074
:1056A00054EFABF060EFABF0010E136E2951030B1A
:1056B000146E1350145E29511418FC0B1418296F22
:1056C0002507D8A0260725512611D8B46AEFABF0DC
:1056D0006CEFABF07AEFABF03FECB7F060008FF41B
:1056E000D9FF600093F4DAFFDF6E0101234B242B16
:1056F00046EFABF0EAECAAF0156E3FECB7F06000B5
:105700008FF4D9FF600093F4DAFFDF6E0101234BC1
:06571000242B15501200CD
:105718003901A3A792EFABF094EFABF0D8EFABF061
:1057280093A799EFABF09BEFABF0D8EFABF06F001E
:10573800A0F7F9F00D0E0001F919D8B4A6EFABF0F7
:10574800A8EFABF0B3EFABF0E45109E1800EE35DF5
:10575800D8A0B1EFABF0B3EFABF0C9EFABF0010EEF
:10576800F46F800EE325D96E030EE421DA6E000E85
:10577800DF6EE3C072F1E4C073F1000EE46F000E57
:10578800E36F39019397D8EFABF0800EE325D96E1C
:10579800030EE421DA6E6000E7F3DFFFE34BE42B4E
:1057A800E3C072F1E4C073F11100000EBA6E000E8E
:1057B800BB6E000EBC6EEF0EC26E9E0EC36E810EE7
:1057C800C46E660E3A01606F610E506F0F0E406F27
:1057D800000E816F000E516F000E416F000E616F59
:1057E800C49ABC9A4099C298C298BA98000E5A6F47
:1057F800000E5B6F000E6A6F000E6B6F000E426F3B
:10580800000E526F180E626F4369536963694469E9
:1058180054696469080E846F090E126F0A0E116FBD
:105828000B0E0D6F0C0E086F140EE26F210E136F26
:10583800220E146F130E166F170EE56F130EE16F1D
:105848001200AC0EF66E6B0EF76E010EF86E00EEDF
:10585800D0F110EE1FF009006F00D7FFEEFFE55002
:10586800E150F9E1A20EF66E6E0EF76E010EF86EBB
:1058780000EEFAF010EE04F009006F00D7FFEEFF1B
:10588800E550E150F9E100EE00F310EE00F1EE6AA8
:10589800E550E150FCE1E250FAE100EE00F2A00E22
:1058A800EE6AE806FDE100EE00F1D00EEE6AE806C9
:1058B800FDE100EED3F0270EEE6AE806FDE15B6A33
:1058C8005A6A596A080ED56E000ED66E000ED76E4B
:1058D800000100EF80F0246E2450F00B0C09256EB7
:1058E80025C01EF05B5056ECB5F016ECB5F0245010
:1058F800F00B0809256E25C01EF05B5056ECB5F07C
:1059080016ECB5F024C022F00F0E22162238F00B48
:105918000C09256E25C01EF05B5056ECB5F016EC50
:10592800B5F024C022F00F0E22162238F00B080919
:10593800256E25C01EF05B5056ECB5F016ECB5F0A0
:105948002404D8A4AAEFACF0ACEFACF0B8EFACF0FC
:10595800090E236E1E0E226EE40EE82EFED7222EAE
:10596800FCD7232EFAD700D01200096E0450051078
:105978000610D8B4C2EFACF0C4EFACF0E5EFACF071
:105988000950030D000EF324D96E010EF420DA6ECF
:10599800600013F0DEFF600017F0DEFF60001BF010
:1059A800DEFF0950020D120EF324D96E010EF42009
:1059B800DA6E60001FF0DEFF600023F0DDFFFFEF0E
:1059C800ACF00950030D000EF324D96E010EF4203B
:1059D800DA6EB20EDE6E6E0EDE6E010EDE6E0950EF
:1059E800020D120EF324D96E010EF420DA6E000EA9
:1059F800DE6E000EDD6E1200000E296E000E286E9F
:105A08001CEFADF028502424266E29502520276E3F
:105A180060009BF0F6FF60009FF0F7FF000EF86E45
:105A28000800F55038ECAEF0284A292A16ECB5F0F3
:105A380028502424266E29502520276E60009BF0CC
:105A4800F6FF60009FF0F7FF000EF86E0800F550B3
:105A58000009D8B432EFADF034EFADF044EFADF05B
:105A68000001FA51285C2950800A266EFB51800AF1
:105A78002658D8A042EFADF044EFADF006EFADF0F8
:105A88001200010129895AEFADF042ECB7F0070E78
:105A980083EFADF00101252915ECB7F0030E83EF74
:105AA800ADF045ECB7F00A0E83EFADF012C10FF080
:105AB80013C110F002D86BEFADF00500FA6E00517B
:105AC800FD6E0151FE6E0251FF6EFA501200116E0A
:105AD800126A1250000AD8B474EFADF055EFADF069
:105AE8001150010AD8B455EFADF0030AD8B449EF04
:105AF800ADF0060AD8B44EEFADF055EFADF0120098
:105B0800246E2450F00B0C09256E25C01EF05B5046
:105B180056ECB5F016ECB5F02450F00B0809256EDC
:105B280025C01EF05B5056ECB5F016ECB5F022041B
:105B3800D8A4A1EFADF0A3EFADF0C1EFADF024C054
:105B480023F00F0E23162338F00B0C09256E25C001
:105B58001EF05B5056ECB5F016ECB5F024C023F0FF
:105B68000F0E23162338F00B0809256E25C01EF0EA
:105B78005B5056ECB5F016ECB5F012003901A3A74E
:105B8800C8EFADF0CAEFADF0CDEFADF06F00A0F704
:105B9800F9F0000E056E000E046E800E0424D96E16
:105BA800030E0520DA6E000EDF6E044A052A055042
:105BB80009E17F0E045CD8A0E4EFADF0E6EFADF0AC
:105BC800D1EFADF03D01F289000EF96F000EFA6FCA
:105BD800000E0301806F000E0101736F000E726FDB
:105BE800000E0001F96F000EF46F3901938D938751
:105BF80012002FECB7F0020E0101286F10EFAEF083
:105C0800FDECB6F037EFAEF055ECB7F037EFAEF08D
:105C1800E7ECB6F037EFAEF014C10FF015C110F095
:105C280020EE03F102D823EFAEF00500FA6EDE5045
:105C3800FD6EDE50FE6EDE50FF6EFA501200116EE1
:105C4800126A1250000AD8B42CEFAEF00CEFAEF086
:105C58001150020AD8B404EFAEF0010AD8B408EF24
:105C6800AEF00CEFAEF01200236E2350F00B0D09CE
:105C78000001E96FE9C01EF05B5056ECB5F016EC78
:105C8800B5F02350F00B09090001E96FE9C01EF0D7
:105C98005B5056ECB5F016ECB5F023C022F00F0EB1
:105CA80022162238F00B0D090001E96FE9C01EF039
:105CB8005B5056ECB5F016ECB5F023C022F00F0E91
:105CC80022162238F00B09090001E96FE9C01EF01D
:105CD8005B5056ECB5F016ECB5F0120060001BF006
:105CE800F6FF60001FF0F7FF000EF86E08006F0067
:105CF800D4FFEAF099EFAEF060001BF0F6FF600009
:105D08001FF0F7FF000EF86E08006F00D4FFEAF0EE
:105D1800600013F0D9FF600017F0DAFF6000ABF302
:105D2800DFFF044A052A064A072A0001EA51D8A4D7
:105D3800A0EFAEF0A2EFAEF080EFAEF0600013F08F
:105D4800D9FF600017F0DAFF000EDF6E120079EC61
:105D5800B1F001012951030B0009D8B4B6EFAEF038
:105D6800B8EFAEF0C5EFAEF0A8ECB6F00009D8B4C5
:105D7800C0EFAEF0C2EFAEF0C5EFAEF0100E01010D
:105D8800276F01012751030D410EF324F66EF80E1B
:105D9800F420F76EF86A000EF82202D8E1EFAEF0B0
:105DA8000500FA6E0900F550FD6E0900F550FE6E0B
:105DB8000900F550FF6EFA5012000101276F12001A
:105DC800000E076E000E066E0DEFAFF03901A3A9A5
:105DD800F0EFAEF0F2EFAEF0EAEFAEF006500424CA
:105DE800D96E07500520DA6EDF503D01EA6F064A8A
:105DF800072A07BE09EFAFF0075009E1810E065CDC
:105E0800D8A009EFAFF00BEFAFF00DEFAFF01BEF3D
:105E1800AFF006500424D96E07500520DA6EDF5023
:105E2800D8A419EFAFF01BEFAFF0EAEFAEF0120015
:105E3800FC0E01012917020E286F29952BEFAFF0F0
:105E480053ECB7F052EFAFF00F0E52EFAFF016C1B0
:105E58000FF017C110F020EE06F102D83EEFAFF0B8
:105E68000500FA6EDE50FD6EDE50FE6EDE50FF6EEF
:105E7800FA501200116E126A1250000AD8B447EF95
:105E8800AFF028EFAFF01150020AD8B424EFAFF00A
:105E9800010AD8B424EFAFF028EFAFF01200B2C077
:105EA80055F0B3C056F0000E0001D46F000ED36F4A
:105EB80071EFAFF0B0C04BF0B1C04CF0550E4D6E65
:105EC800000E4E6EB4C04FF0B5C050F08DEC8CF0A3
:105ED8004B500001D3274C50D423600057F1F6FFF4
:105EE80060005BF1F7FF000EF86E0800F55000093E
:105EF800D8A481EFAFF083EFAFF05EEFAFF0D3C07F
:105F0800B0F0D4C0B1F012000AC00EF00BC00FF010
:105F180008C010F009C011F00E500C6E0F500D6E35
:105F28000E4A0F2A600033F0F6FF600037F0F7FFE3
:105F3800000EF86E600043F0D9FF600047F0DAFF0A
:105F4800104A112A1F0EF76403D00800F55007D035
:105F58006F00DBFFE9FF6F00DFFFEAFFEF50DF6E46
:105F6800DF50D8A4BAEFAFF0BCEFAFF090EFAFF0CE
:105F78001200000E286E000E276ED0EFAFF02750EB
:105F88002424D96E28502520DA6EDF5038ECAEF084
:105F980016ECB5F0274A282A27502424D96E285011
:105FA8002520DA6EDF50D8B4DCEFAFF0DEEFAFF0CB
:105FB800EEEFAFF00001FA51275C2850800A266EF8
:105FC800FB51800A2658D8A0ECEFAFF0EEEFAFF007
:105FD800C3EFAFF012001D6E1D5098ECAAF0000937
:105FE800D8B4F9EFAFF0FBEFAFF0F0EFAFF019C0B6
:105FF80004F01AC005F01BC006F01CC007F0A3ECA3
:10600800B5F0000E0A6E000E0B6E000E0C6E000E40
:106018000D6E000E0E6E20ECB6F01FECB7F000EC23
:10602800B5F0E806D8B41BEFB0F01DEFB0F013EFF1
:10603800B0F01200000E3E01DE6F000EDF6F000EA2
:10604800E06F000EE16F000EE46F000EE56F000ECA
:10605800EA6F000EEC6F000EF16F000EF36F000E8A
:10606800F46F000EF56F000EF66F000EF76F000E5E
:10607800F96F000EFA6F000EFB6F000EFC6F000E3A
:10608800FD6F000EFE6F030EFF6F840EF86F120097
:106098003901A3A152EFB0F054EFB0F056EFB0F0D1
:1060A80079EFB0F0A2AF5BEFB0F05DEFB0F05FEF6B
:1060B800B0F079EFB0F03D0179A565EFB0F067EF8A
:1060C800B0F069EFB0F079EFB0F079AF6EEFB0F003
:1060D80070EFB0F072EFB0F079EFB0F076A977EF2B
:1060E800B0F079EFB0F04CEFB0F012006F00E8FFBD
:1060F80001F06F00ECFF02F03901A39F0001FF518E
:10610800B76E6000FBF3B6FF0101F351F411F5110E
:10611800D8B491EFB0F093EFB0F0A0EFB0F002D8A0
:10612800A0EFB0F00500FA6EF351FD6EF451FE6E6B
:10613800F551FF6EFA50120060000BF0FBFF600093
:1061480007F0FAFF110004C006F005C007F0AFEF32
:10615800B0F0044A052A600013F0F6FF600017F05B
:10616800F7FF000EF86E1F0EF76403D00800F55015
:1061780007D06F00DBFFE9FF6F00DFFFEAFFEF509A
:106188000009D8A4CAEFB0F0CCEFB0F0ADEFB0F092
:106198000650045C046E07500558056E1200EBEFBC
:1061A800B0F03901A3A9DBEFB0F0DDEFB0F0D5EF27
:1061B800B0F0600013F0F6FF600017F0F7FF000E74
:1061C800F86E08006F00D7FFEAFD044A052A600050
:1061D80013F0F6FF600017F0F7FF000EF86E0800E6
:1061E800F5500009D8A4FBEFB0F0FDEFB0F0D5EF03
:1061F800B0F01200BA0E0001C26F000EC36FB6C035
:10620800C4F0B7C0C5F0000EC86F000EC76F000E0F
:10621800CE6F000ECD6FC40EB06F000EB16FB8C058
:10622800B2F0B9C0B3F0C20EB46F000EB56F53EC44
:10623800AFF00001C751B625D96EC851B721DA6E43
:10624800000EDF6E1200010E0A6E200E04180510F3
:10625800D8B431EFB1F033EFB1F04CEFB1F0F70E45
:10626800066EFF0E076E04C008F005C009F0065060
:10627800082607500922095009E1050E085CD8A034
:1062880048EFB1F04AEFB1F04CEFB1F0000E0A6EF2
:106298000AC004F0056A1200176E010E186E01019B
:1062A80029B559EFB1F05BEFB1F077EFB1F029857F
:1062B800000E186E255115ECB7F01750D8B467EFDB
:1062C800B1F069EFB1F070EFB1F0040E0101276F82
:1062D800E9ECB4F075EFB1F0030E0101276F92EC11
:1062E800B6F0E6ECB5F018501200D4ECB6F00009A0
:1062F800D8B481EFB1F083EFB1F087EFB1F04EEC95
:10630800B7F0A1EFB1F0BEECB6F00009D8B48FEF4A
:10631800B1F091EFB1F095EFB1F048ECB7F0A1EF23
:10632800B1F0C9ECB6F00009D8B49DEFB1F09FEF19
:10633800B1F0A1EFB1F04BECB7F0120020EE02F093
:106348000F50D9261050DA226F0078FF04F06F0042
:1063580074FF05F060003FF0D9FF600043F0DAFFFA
:106368006F0078FF06F06F0074FF07F0A3ECB5F03C
:10637800000E0A6E000E0B6E000E0C6E000E0D6EF7
:10638800000E0E6E2EECB6F0020E1200000E3D014D
:10639800EC6F000EED6F000EEE6F000EEF6F000E4B
:1063A800F06F000EF16FB00EF26F800EF36F000EFB
:1063B800F46F8A0EF56F000EF66F000EF76F000E81
:1063C800F86F000EF96F000EFA6FF28BF28939013F
:1063D80093971200BF0E0C6EFF0E0D6E0AC00EF0E2
:1063E8000BC00FF00C500E260D500F220F5007E176
:1063F8001A0E0E5CD8B003EFB2F005EFB2F00CEF56
:10640800B2F0200E0A100A6E0B500B6E10EFB2F0AD
:106418000AC00AF00BC00BF01200000E211A000E81
:10642800221A000E231A800E241A1DC004F01EC062
:1064380005F01FC006F020C007F021C008F022C0F8
:1064480009F023C00AF024C00BF06BEC92F004C0F2
:106458001DF005C01EF006C01FF007C020F0120096
:10646800056E800E066E4EEFB2F005500614000958
:10647800D8B441EFB2F043EFB2F048EFB2F02A0ED1
:10648800C6ECB5F04BEFB2F0200EC6ECB5F0D890E4
:106498000630066E0650D8A454EFB2F056EFB2F0AC
:1064A80039EFB2F012009F0E0C6EFF0E0D6E0AC08F
:1064B8000EF00BC00FF00C500E260D500F220F508F
:1064C80007E11A0E0E5CD8B06CEFB2F06EEFB2F0C6
:1064D80074EFB2F05F0E0A140A6E0B6A78EFB2F02E
:1064E8000AC00AF00BC00BF01200000E136E000E6B
:1064F800126E8AEFB2F011C004F0056A0FC006F000
:1065080010C007F08AECA7F0124A132A12500D2483
:10651800D96E13500E20DA6EDF50116E1150D8A4C8
:1065280098EFB2F09AEFB2F07FEFB2F01200430E9C
:10653800B96EEB0EB76E000EB66EB6506F00DCFE8D
:1065480007F0086A07C008F0076A07100001FE6F25
:106558000850FF6F3901A39F938FBA0E046E6E0E19
:10656800056E010E066EEFECB6F0900EB86E1200D6
:10657800D29ED28AD29ED29CD28A550ED46EAA0EB0
:10658800D46ED490000ED76E000ED66E080ED56E5F
:10659800550ED46EAA0ED46ED480390183878181BA
:1065A8008491839F8495809FD29CD29ED29E120014
:1065B80017BEE9EFB2F0175006E11604D8B0E7EFBE
:1065C800B2F0E9EFB2F0F7EFB2F016C018F017C06A
:1065D80019F0181E191E184A192A18C016F019C0E1
:1065E80017F0FBEFB2F016C016F017C017F0120044
:1065F800066E000E0001EB6F10EFB3F0520E056E41
:106608002B0E046E000EE82EFED7042EFCD7052EA6
:10661800FAD700D00001EB2B0650EB5DD8A017EF9E
:10662800B3F019EFB3F002EFB3F012009F0E066E4D
:10663800FF0E076E200E0410086E000E0510096E7E
:10664800065008260750092209500AE11A0E085C6C
:10665800D8A031EFB3F034EFB3F0010E35EFB3F05B
:10666800000E046E056A12006F0060FF03F000015F
:10667800DD51DE11D8B443EFB3F045EFB3F04AEF84
:10668800B3F0DD07D8A0DE074DEFB3F0ED8B39018D
:106698009991010E0001F06F3901A99160000FF086
:1066A800D8FF11009F0E066EFF0E076E04C008F09B
:1066B80005C009F0065008260750092209500AE1CA
:1066C8001A0E085CD8A06BEFB3F06EEFB3F0010EB2
:1066D8006FEFB3F0000E046E056A1200BF0E066E6F
:1066E800FF0E076E04C008F005C009F00650082622
:1066F8000750092209500AE11A0E085CD8A087EF52
:10670800B3F08AEFB3F0010E8BEFB3F0000E046E16
:10671800056A12000450051006100710D8B497EF48
:10672800B3F099EFB3F0A1EFB3F0000E041A000E26
:10673800051A000E061A800E071A04C004F005C0D8
:1067480005F006C006F007C007F01200D00E066E6E
:10675800FF0E076E04C008F005C009F006500826B1
:106768000750092209500AE10A0E085CD8A0BFEFB9
:10677800B3F0C2EFB3F0010EC3EFB3F0000E046E36
:10678800056A1200390191A1CCEFB3F0CEEFB3F056
:10679800DAEFB3F0A1A1D3EFB3F0D5EFB3F0DAEFAE
:1067A800B3F00001ED9F230E3D01EA6F3901A09F70
:1067B800000E3A01576F3901A19111003D017995F9
:1067C800600013F06EFD000E6C6F738B79A5EFEF10
:1067D800B3F0F1EFB3F0EAEFB3F074ABF6EFB3F068
:1067E800F9EFB3F0010EFAEFB3F0000E1200FF0E4E
:1067F8000416030E051672A804EFB4F006EFB4F001
:106808000DEFB4F0060ED89004360536E82E07EFE3
:10681800B4F00550716E600013F070FF1200FF0EA7
:106828000416030E051676A81CEFB4F01EEFB4F09C
:1068380025EFB4F0060ED89004360536E82E1FEF83
:10684800B4F00550756E600013F074FF1200FF0E6F
:106858000416030E05167AA834EFB4F036EFB4F038
:106868003DEFB4F0060ED89004360536E82E37EF23
:10687800B4F00550796E600013F078FF1200FF0E37
:106888000416030E05167EA84CEFB4F04EEFB4F0D4
:1068980055EFB4F0060ED89004360536E82E4FEFC3
:1068A800B4F005507D6E600013F07CFF12000FC03D
:1068B80004F010C005F0000E076E010E066EA3EC82
:1068C800B5F0000E0A6E000E0B6E000E0C6E000E78
:1068D8000D6E000E0E6E2EECB6F0040E12000FC0F8
:1068E80004F010C005F0000E076E020E066EA3EC51
:1068F800B5F0000E0A6E000E0B6E000E0C6E000E48
:106908000D6E000E0E6E2EECB6F0020E12000FC0C9
:1069180004F010C005F0000E076E010E066EA3EC21
:10692800B5F0000E0A6E000E0B6E000E0C6E000E17
:106938000D6E000E0E6E2EECB6F0020E12000FC099
:1069480004F010C005F0000E076E020E066EA3ECF0
:10695800B5F0000E0A6E000E0B6E000E0C6E000EE7
:106968000D6E000E0E6E2EECB6F0040E12003901FC
:10697800A3A9C1EFB4F0C3EFB4F0BBEFB4F00D0EB0
:106988003D01EA6F3901A3A9CCEFB4F0CEEFB4F022
:10699800C6EFB4F00A0E3D01EA6F12003D0173BF65
:1069A800D8EFB4F0DAEFB4F0E8EFB4F0000E796F96
:1069B800000E7A6F000E766F6C69510E3A016A6F9D
:1069C800510E6B6F3D01738F120001012951FC0BB1
:1069D8000209296F25052611D8A4F5EFB4F0F7EFC1
:1069E800B4F0F9EFB4F0EAECAAF0D880010122354E
:1069F80010ECB7F0040E1200010E046E010129B567
:106A080008EFB5F00AEFB5F014EFB5F02997226951
:106A18002FECB7F0F5ECB5F00AECB7F028C104F0AC
:106A280004501200000E056E000E046E00F0044AB9
:106A3800052A05BE29EFB5F0055009E1A00E045C52
:106A4800D8A029EFB5F02BEFB5F01AEFB5F012008A
:106A5800045006026F00CCFF08F06F00D0FF09F069
:106A680004500702F350092605500602F350092680
:106A780008C004F009C005F0120091ECB5F086ECEE
:106A8800B6F06EECB6F01EECB0F004ECB6F056ECD6
:106A9800B6F012ECB6F09BECB2F07AECB6F062EC21
:106AA800B6F012001F6E1EC020F0000E216E200EE0
:106AB800196E000E1A6E000E1C6E010E1B6E1F5012
:106AC800EFECAFF0A00EE82EFED7120036ECB7F0D0
:106AD80033ECB7F00009D8B474EFB5F076EFB5F041
:106AE8007CEFB5F0000E15ECB7F0000E10ECB7F027
:106AF800000E120012C004F013C005F0A7ECB0F0AD
:106B080004501224086E05501320096E14C00AF0B0
:106B180015C00BF088ECAFF01200000E3901C06F01
:106B2800000EC16F000EC26F000EC36F000EC46F5F
:106B3800000EC56F1D0EC66F030EC76F1200010150
:106B480029A9A9EFB5F0ABEFB5F0B4EFB5F004C0E3
:106B580023F105C024F106C025F107C026F12999C3
:106B68001200030E3D017B6F040E736F800E746F6D
:106B7800000E756F000E6C6F7599200E6E6F79950B
:106B8800739F1200046ECAEFB5F000F03901A3A993
:106B9800D0EFB5F0D2EFB5F0C9EFB5F0600013F063
:106BA800EAFD120072FA37FAD4FAFBFA1EFBFFF874
:106BB800FBF980F982F8BEF952FBAAFA286E756CC7
:036BC8006C290035
:106BCC00ECEFB5F04CECB0F0ABECAEF0010129B54C
:106BDC00F2EFB5F0F4EFB5F0E8EFB5F012003901D3
:106BEC0093939395929F93913D017A917A957A9F85
:106BFC007A9D7A937693769576911200010EA26E19
:106C0C00000EA16E000EA36E9F68000E9E6E3901E1
:106C1C00A791C00EA06E1200010EAE6E000EAD6EEE
:106C2C00000EAF6EAB68000EAA6E3901A495C00EB3
:106C3C00AC6E12000AC004F00BC005F00CC006F0DC
:106C4C000DC007F00EC008F0020EB9ECACF012004B
:106C5C000AC004F00BC005F00CC006F00DC007F024
:106C6C000EC008F0000EB9ECACF012002E6E2BC06A
:106C7C0026F02E508FECA9F02CC024F02DC025F05E
:106C8C00BDECAFF012002E6E2BC026F02E508FEC08
:106C9C00A9F02CC024F02DC025F000ECADF01200B2
:106CAC008C0E726E000E716E000E706E3F015E5196
:106CBC003F0B80095E6F12008C0E766E000E756EA7
:106CCC00000E746E3F015E51CF0B20095E6F1200F7
:106CDC008C0E7A6E000E796E000E786E3F015E514E
:106CEC00F30B08095E6F12008C0E7E6E000E7D6E2B
:106CFC00000E7C6E3F015E51FC0B01095E6F1200B1
:106D0C00600E3901D96F000EDB6F000EDD6F080EBF
:106D1C00DF6F000EDE6F120001012951FC0B02091E
:106D2C00296F2251222510ECB7F0030E12003D0101
:106D3C0078BBA3EFB6F0A6EFB6F0010EA7EFB6F056
:106D4C00000E12003D0174BBAEEFB6F0B1EFB6F021
:106D5C00010EB2EFB6F0000E12003D0178B1B9EFA2
:106D6C00B6F0BCEFB6F0010EBDEFB6F0000E12009F
:106D7C003D0179B5C4EFB6F0C7EFB6F0010EC8EF20
:106D8C00B6F0000E12003D0176B9CFEFB6F0D2EF9F
:106D9C00B6F0010ED3EFB6F0000E12003D0179BF34
:106DAC00DAEFB6F0DDEFB6F0010EDEEFB6F0000E66
:106DBC0012001AECB7F001012995020E286F0F0E84
:106DCC0012001AECB7F001012995000E286F0F0E76
:106DDC00120004C0F3F105C0F4F106C0F5F1120085
:106DEC0039ECB7F036ECB7F004ECB7F01200010157
:106DFC00255115ECB7F0E9ECB4F01200010129951E
:106E0C00000E286F0F0E12003D01739F000E796F5C
:106E1C0078851200046E600013F06BFD1200046E96
:106E2C00600013F06CFD12003D01739F7885738F29
:106E3C001200000E50ECB1F0120039ECB7F0090E54
:106E4C0012003CECB7F0040E12003CECB7F0030E51
:106E5C001200000E3D01796F12003D016C511200C1
:106E6C003D01739B12003D01748D12003D01749D18
:106E7C0012003D016A5112003D01738D12003D015B
:106E8C00739D12003D01799512003D017699120017
:106E9C003D01799F120014002020010E1200020EF9
:106EAC001200050E1200010E120012001100120049
:020000040020DA
:10000000FFFFFFFFFFFFFFFFFFFFFFFFFFFFFFFF00
:020000040030CA
:0A0000008CFFFFFF9FFFFFFFFFFFD3
:00000001FF
